:100000000C941E060C94A0280C94CD280C94460643
:100010000C9446060C94E9120C9446060C94460681
:100020000C9446060C9446060C9446060C94460620
:100030000C9446060C9446060C9446060C94460610
:100040000C94FA280C9446060C94E82C0C942B2D56
:100050000C9446060C9446060C9446060C944606F0
:100060000C9446060C944606F8185A1939193C198E
:100070003F194219451948194B195A1954198C1A24
:100080008E1A8E1A8C1A8E1A8E1A8E1A8E1A8E1A32
:100090008E1A8E1A8E1A8E1A8E1A8E1A8E1A8E1A20
:1000A000121A8E1A8E1A8E1A8E1A8E1A83198E1A98
:1000B0008E1A8E1A8E1A8E1A8E1A8E1A8E1A8E1A00
:1000C0008E1A8E1A8E1A8E1A8E1A8E1A1E1A1E1AD0
:1000D0001E1A1E1A1E1A1E1A1E1A1E1A1E1A8E1AF0
:1000E0008E1A8E1A8E1A8E1A8E1A83191D1A1D1ABE
:1000F0001D1A1D1A8E1A2B1A311A371A3D1A431A55
:10010000491A4F1A551A5F1A691A731A7D1AC419B7
:1001100086198E1A8E1A8E1A8E1A121A8E1A8E1A24
:100120008E1A8E1A8E1A8E1A8E1A8E1A1C1A1C1A73
:100130001C1A1C1A8E1A2B1A311A371A3D1A431A16
:10014000491A4F1A551A5F1A691A731A7D1AC41977
:1001500086198E1A8E1A8E1A8E1A121AC11AC11A7E
:10016000C11AC11AC11AC11AC11AC11AC11AC11AB7
:10017000C11AC11AC11AD81BD81BD81BD81BD81B2F
:10018000D81B061B101B1A1B241B821B8C1B9B1BC2
:10019000AC1B341D491D551D5E1D6D1D921D9B1D03
:1001A000E41DAD1DF920FF2005210C211A213C2161
:1001B0005A21456E746572206D656E752E2E2E0067
:1001C000546F67676C6564206D6963726F50504D42
:1001D00000546F67676C656420696E76657274653C
:1001E000642050504D2100546F67676C6564205443
:1001F00058206D7574696E672100546F67676C6570
:10020000642074656C656D65747279210050726F3D
:10021000746F636F6C206572726F72207769746897
:100220002052580054696D656F7574207768656E4B
:1002300020636F6E6E656374696E6720746F205201
:100240005800507265737320616E79206B65792058
:10025000746F2063616E63656C00436F6E6E6563DF
:1002600074696E6720746F2052582C20706F776508
:100270007220757020746865205258202877697440
:10028000682062696E6420706C7567206966206EF4
:100290006F74207573696E6720616C776179732064
:1002A00062696E642900546F67676C656420276912
:1002B0006D6D656469617465206F75747075742700
:1002C00000546F67676C65642027736C61766520E6
:1002D0006D6F64652700546F67676C6564202761E4
:1002E0006C776179732062696E642700546F676769
:1002F0006C65642050504D206368616E6E656C20A3
:100300006C696D69740053657420525353492069B8
:100310006E6A656374696F6E206368616E6E656C8A
:100320002028303D3D64697361626C652900536526
:10033000742050504D206D696E696D756D20737914
:100340006E630053657420626561636F6E20696E31
:1003500074657276616C0053657420626561636FC9
:100360006E2064656C617900536574206265616319
:100370006F6E206672657175656E637920696E2097
:10038000487A3A20303D64697361626C652C205074
:10039000783D504D52206368616E6E656C20782CFC
:1003A0002046783D465253206368616E6E656C202E
:1003B00078005365742050574D2073746F7020641B
:1003C000656C61792028302064697361626C6564B2
:1003D0002C20312D323535203D3D20302E317320FB
:1003E0002D2035306D696E29005365742050504DB5
:1003F0002073746F702064656C61792028302064EC
:10040000697361626C65642C20312D323535203D75
:100410003D20302E3173202D2035306D696E29003E
:10042000536574206661696C736166652064656CF0
:1004300061792028302064697361626C65642C20C6
:10044000312D323535203D3D20302E3173202D2089
:1004500035306D696E29002A2A2A2A2A2A2A2A2A50
:100460002A2A2A2A2A2A2A2A2A2A2A2A2A2A2A2AEC
:100470002A2A2A2A0052582041636B6564202D20C5
:1004800072657665727420737563636573736675E0
:100490006C21002A2A2A2A2A2A2A2A2A2A2A2A2AAD
:1004A0002A2A2A2A2A2A2A2A2A2A2A2A2A2A2A2AAC
:1004B000002A2A2A2A2A2A2A2A2A2A2A2A2A2A2AC6
:1004C0002A2A2A2A2A2A2A2A2A2A2A2A2A2A00528E
:1004D000582041636B6564202D20757064617465DC
:1004E000207375636365737366756C21002A2A2A0D
:1004F0002A2A2A2A2A2A2A2A2A2A2A2A2A2A2A2A5C
:100500002A2A2A2A2A2A2A2A2A2A0056616C696457
:100510002063686F69636573206172653A205B319F
:100520005D2D5B31365D20286368616E6E656C20E1
:10053000312D31362900536574206F7574707574D0
:1005400020666F7220706F727420005B585D2061AE
:10055000626F7274206368616E67657320616E6498
:10056000206578697420525820636F6E6669670051
:100570005B535D20736176652073657474696E6783
:100580007320746F205258005B525D20726576654F
:1005900072742052582073657474696E6773207486
:1005A0006F2064656661756C747300557365206EA9
:1005B000756D62657273205B312D445D20746F2010
:1005C0006564697420706F727473205B452D515D92
:1005D00020666F722073657474696E677300202DD6
:1005E00020726563656976657220636F6E66696700
:1005F000757261746F722C20727820737720000AF4
:100600000A6F70656E4C52536E67200053657420FC
:1006100073657269616C2062617564726174653AB8
:10062000200056616C69642063686F696365733A82
:100630002031202D20342B34202F2032202D203823
:10064000202F2033202D20382B34202F2034202D14
:10065000203132202F2035202D2031322B34202FF5
:100660002036202D20313600536574204368616E9A
:100670006E656C20636F6E6669673A20005365741F
:100680002044617461726174652028302D32293AEA
:10069000200053657420486F70206368616E6E653A
:1006A0006C7320286D61782032342C207365706162
:1006B000726174656420627920636F6D6D61732966
:1006C0002076616C69642076616C75657320312DCC
:1006D0003235353A2000536574206368616E6E656B
:1006E0006C2073706163696E6720287831306B48C5
:1006F0007A293A200053657420524620706F77653E
:10070000722028302D37293A200053657420524634
:10071000206D6167696320286865782920652E67E8
:100720002E20307844454144463030443A2000532E
:1007300065742062617365206672657175656E63AC
:10074000792028696E20487A293A20005B5A5D207A
:10075000656E746572207265636569766572206383
:100760006F6E66696775726174696F6E2075746902
:100770006C79005B465D20646973706C61792061FF
:10078000637475616C206672657175656E63696509
:10079000732075736564005B525D2063616C6375E3
:1007A0006C6174652072616E646F6D206B65792079
:1007B000616E6420686F70206C697374005B495DC2
:1007C000207265696E697469616C697A6520736508
:1007D0007474696E677320746F20736B65746368DB
:1007E0002064656661756C7473005B585D2072658A
:1007F00076657274206368616E67657320616E64EC
:100800002065786974206D656E75005B535D20739B
:100810006176652073657474696E677320746F20E8
:10082000454550524F4D20616E64206578697420B3
:100830006D656E7500557365206E756D62657273BA
:10084000205B302D395D20746F20656469742070E1
:100850006172616D657465727300202D2053797328
:1008600074656D20636F6E66696775726174696F18
:100870006E000A0A6F70656E4C52536E672000510D
:1008800029204F7574707574206265666F726520DB
:100890006C696E6B20283D465329203A2000502970
:1008A00020536C617665206D6F64652028657870D3
:1008B0006572696D656E74616C293A20004F29205C
:1008C00054696D65642042494E44206174207374FC
:1008D000617274757020203A20004E292050504DCE
:1008E000206F7574707574206C696D69746564200F
:1008F000202020203A200044495341424C454400E6
:100900004D292050504D205253534920746F20637D
:1009100068616E6E656C202020203A20004C2920F2
:1009200050504D206D696E696D756D2073796E63E1
:10093000202875732920203A200044495341424C15
:100940004544004B29204661696C736166652062ED
:100950006561636F6E20696E74762E2028312D32AA
:10096000353573293A20004A29204661696C736144
:10097000666520626561636F6E2064656C617920D5
:1009800028302D323535203D3E20313073202D204A
:100990003135306D696E293A200049292046616958
:1009A0006C7361666520626561636F6E206672714B
:1009B0002E203A200048292050574D2073746F7024
:1009C0002064656C6179202020202020203A2000BE
:1009D00047292050504D2073746F702064656C61FE
:1009E00079202020202020203A200046292046611E
:1009F000696C736166652064656C617920202020D4
:100A00002020203A200050574D206368616E6E65AB
:100A10006C200066756E6374696F6E3A2000292041
:100A2000706F72742000506F776572546F776572C3
:100A300000445446205548462033322D62697420C4
:100A400031306368004F70656E4C52536E67525878
:100A5000206D696E6920342F36636800466C7974A6
:100A6000726F6E2F4F72616E6765525820554846FF
:100A70002038636800525820747970653A20004429
:100A8000697361626C656400487A00203D3D200016
:100A900043616C63756C61746564207061636B6540
:100AA0007420696E74657276616C3A200042292068
:100AB0004D6963726F202868616C66292050504D23
:100AC000202020203A00412920496E766572746505
:100AD000642050504D20696E20202020203A0030A4
:100AE00029204D7574652062757A7A657220286DAB
:100AF0006F73746C79293A003929205365726961E2
:100B00006C2062617564726174653A00736D617224
:100B100074506F7274004672536B79005472616E38
:100B200073706172656E740044697361626C6564B0
:100B30000038292054656C656D657472793A2020FF
:100B40002020202020003729204368616E6E656CCC
:100B500020636F6E6669673A202000362920446161
:100B60007461726174652028302D32293A2020206A
:100B700000352920486F70206368616E6E656C7364
:100B80003A2020202020003429204368616E6E65C1
:100B90006C2073706163696E673A202000332920EE
:100BA000524620706F7765722028302D37293A2001
:100BB0002020003229205246206D616769633A2067
:100BC0002020202020202020003129204261736530
:100BD000206672657175656E63793A202020000089
:100BE00000000700020100000304060000000000EE
:100BF00000000001020408102040800102040810D7
:100C00002001020408102004040404040404040263
:100C10000202020202030303030303000000002395
:100C2000002600290000000000250028002B0000FD
:100C3000000000240027002A0000192E11241FBEE6
:100C4000CFEFD8E0DEBFCDBF13E0A0E0B1E0E0E43D
:100C5000F2E602C005900D92A83CB107D9F716E064
:100C6000A8ECB3E001C01D92A039B107E1F71CE088
:100C7000CCE3DCE004C02297FE010E94222FCA339D
:100C8000D107C9F70E94552E0C941E310C94000018
:100C900080917505813019F482E08093750580910B
:100CA0007505833019F484E0809375050895A8953F
:100CB0000895DC01ED91FC910190F081E02D099502
:100CC00008952091760530917705382748E0C901CD
:100CD000880F991F37FF06C09C0151E2252750E17C
:100CE000352701C09C01415091F73093770520933F
:100CF0007605089588E38093780580E092ECA1E082
:100D0000B0E08093790590937A05A0937B05B0932A
:100D10007C0587E08093850580EC9AECA9E8B6E332
:100D200080937D0590937E05A0937F05B093800509
:100D300085E0809386058DEE9EEFADEABEED809353
:100D4000810590938205A0938305B0938405E7E81D
:100D5000F5E080E090E0863028F4DC01AE54BC4F32
:100D60002C9101C020E0219301968831910599F7DB
:100D700082E080939F058AE08093A005089580EC2F
:100D800097EFAAEBB7E38093BD059093BE05A093C0
:100D9000BF05B093C00580E090E0A0E0B0E580938F
:100DA000C1059093C205A093C305B093C405E5ECBB
:100DB000F5E080E081938F5F8031E1F70895A0E056
:100DC000B0E0E5EEF6E00C94EB2ED82F0E9450290F
:100DD0006115710581059105C9F30E948E2F10924E
:100DE0008105109282051092830510928405C4E05B
:100DF000812C912C54018A94C0908105D090820559
:100E0000E0908305F0908405FE2CED2CDC2CCC24A6
:100E10000E94892FA50194010E94CA2E6C0D7D1D90
:100E20008E1D9F1D609381057093820580938305BD
:100E300090938405C15001F7DD2309F450C007E801
:100E400015E0E801A12CB12C62E3C62ED12CE12CD7
:100E5000F12C8881882309F442C0B39419F40E94CC
:100E60007A063DC00E94892FA70196010E94CA2ED2
:100E7000E1E0E60FA7E8B5E08A2F801B8A1520F491
:100E80008D918E13F9CFE9CF2091860530E0A0E156
:100E9000B7E20E94622E9B01AC01AE2FB0E00E942F
:100EA000712E40907D0550907E0560907F0570907A
:100EB0008005640D751D861D971D4090BD055090E1
:100EC000BE056090BF057090C005461657066806BF
:100ED000790618F2E993A39488E1A812BACFCDB7A6
:100EE000DEB7E0E10C94072F8436910520F4BC01B5
:100EF00080E090E017C09C018E3B910528F42A55B4
:100F00003109AAE0B0E00CC0823D910528F4245BD1
:100F10003109A4E6B0E004C02D5C3109A8E5B2E0D7
:100F20000E94622EA4E6B0E09B01AC010E94712EEB
:100F3000089590E08C599F4F0E947407089561E0D6
:100F40008AE00E94FD2960E08AE00E94362A089526
:100F5000892B11F061E001C060E08AE00E94362A2E
:100F6000089560E089E00E94FD2961E088E00E9428
:100F7000FD2961E087E00E94FD2960E082E00E9497
:100F8000FD2961E084E00E94FD29089542E050E0DF
:100F900068E476E080E00E9480280895E3E0F0E0D5
:100FA00089E080935700E491E67081E0E63009F033
:100FB00080E00895CF93DF93C82F0E94CE07882347
:100FC00081F0DFB781E080937405F8940E945706A2
:100FD00088E180936000C0936000C1110E945706B1
:100FE000DFBFDF91CF9108958F929F92AF92BF9212
:100FF000CF92DF92EF92FF92CF93FC01C0A5EC2F2E
:10100000E770F0E0E658FC4FA081B0E0C7FF03C0F6
:1010100024E130E002C02FE030E0FC0197A183E141
:10102000989FF0011124E25CFE4F80809180A280A5
:10103000B380A20FB31F20E43FE14DE750E00E94D0
:101040007C2EA50194010E94A82E8C2F887149F452
:1010500069017A01E0EDCE0EE7E0DE1EE11CF11C35
:101060001BC0C7FF05C060E47AE88CE29EE004C0C4
:1010700060E07EEE8AEB9BE069017A01F8EBCF0E2F
:10108000FBE0DF1EE11CF11CA50194010E94A82ECB
:10109000C20ED31EE41EF51EC701B60169517C4F76
:1010A0008F4F9F4F28EE33E040E050E00E94A82E83
:1010B000A8EEB3E00E94712ECF91FF90EF90DF90E9
:1010C000CF90BF90AF909F908F9008958F3F9105E4
:1010D00051F048F0811522E0920738F081159340D5
:1010E00030F482E0089580E0089581E0089583E07F
:1010F0000895A0E0B0E0EFE7F8E00C94F42EEB01E7
:101100008A01B82FB695A0E028813981F8012083A3
:101110002A813B8121832C813D8122832E813F8145
:101120002383688179814A815B812C813D81EE81B5
:10113000FF819F2F9295990F990F907C272F2370F5
:10114000922B252F2370220F220F922B232F2370F7
:101150002295207F922BF80194830B5F1F4F2896D6
:10116000AF5FBA1788F680FF24C0888199810E94FA
:101170006608D82E8A819B810E946608E82E8C81A1
:101180009D810E946608F82E8E819F810E946608CC
:10119000F0E4DF9EA001112490E1E99E900111246A
:1011A000242B282BE4E0FE9EB0011124262BF8010D
:1011B0002083CDB7DEB7E7E00C94102F803223E018
:1011C000920708F1883E23E0920740F48F51934044
:1011D000E4E096958795EA95E1F70895803D27E04C
:1011E000920718F48C5D93400895883928E092079F
:1011F00068F4885C974074E0969587957A95E1F756
:101200008D509C4F089580E090E008958FEF93E01B
:1012100008958C30910540F4A4E0880F991FAA9599
:10122000E1F7885D9C4F0895843F23E0920718F40E
:1012300084529C4F0895811524E0920740F486570C
:10124000934FF4E0880F991FFA95E1F7089580E92C
:1012500098E008959C013695279525753575821B74
:10126000930B9C0123733373969587959695879579
:1012700083739373820F931F9C0154E036952795D7
:101280005A95E1F7280F391F2F703F7041E051E068
:10129000249FC001259F900D349F900D1124892F0C
:1012A00008955F98882319F00000289A02C0000072
:1012B000289800005F9A000008955F9A000083B1AB
:1012C0005F980000869581700895CF93DF93D82FA3
:1012D0005C9A5F985C98C8E08D2F80780E945109D5
:1012E000DD0FC150C9F75F98DF91CF9108958F77D7
:1012F0000E9465090895CF93DF93D82FC8E08D2F02
:1013000080780E945109DD0FC150C9F75F98DF91C5
:10131000CF910895CF93DF935F98C8E080E0D82FF6
:10132000DD0F0E945D098D0FC150C9F7DF91CF918C
:1013300008950E9477090E948A095C9A0895A1E0A5
:10134000B0E0E5EAF9E00C94F92E806869830E9428
:1013500065096981862F0E947B095C9A2196E2E0EB
:101360000C94152FCF93C0918105C827E82FF0E08A
:10137000E858FA4F678589E70E949F096C2F8DE333
:101380000E949F096C2F82E40E949F09CF910895CB
:1013900086E20E9499090895CF93DF93EC016C8156
:1013A0008CE10E949F096D818DE10E949F096E81F1
:1013B0008EE10E949F096F8180E20E949F096885EB
:1013C00081E20E949F09698582E20E949F096A85E5
:1013D00083E20E949F096B8584E20E949F096C85CD
:1013E00085E20E949F096D858AE20E949F096E85B1
:1013F0008EE60E949F096F858FE60E949F0968898B
:1014000080E70E949F09698981E70E949F096A8994
:1014100082E70E949F09DF91CF910895CF92DF92DA
:10142000EF92FF92CF93DF936B017C01C11488E3AD
:10143000D8068CE9E8068CE1F80628F5C701B60164
:1014400020E836E948E950E00E94A82EE9016897B3
:1014500060E879E687E69FEF0E94842E6C0D7D1D83
:101460008E1D9F1DF2E0660F771F881F991FFA954A
:10147000D1F721E732E040E050E00E94A82EF22EA2
:10148000E32E80E421C0C701B60120E03DE241E344
:1014900051E00E94A82EE901689760E073ED8EECA0
:1014A0009EEF0E94842E6C0D7D1D8E1D9F1D660F6C
:1014B000771F881F991F21E732E040E050E00E942B
:1014C000A82EF22EE32E80E66C2F6F71680F85E751
:1014D0000E949F096E2D86E70E949F096F2D87E766
:1014E0000E949F09DF91CF91FF90EF90DF90CF9006
:1014F0000895682F8DE60E949F0908958F929F920C
:10150000AF92BF92CF92DF92EF92FF92CF93DF9391
:10151000D82F83E00E9499098093730584E00E948C
:1015200099098093720560E086E00E949F0961E05E
:1015300087E00E949F096FE789E00E949F0965E0AC
:101540008AE00E949F0962E18BE00E949F0965E1A9
:101550008CE00E949F096DEF8DE00E949F0960E082
:101560008EE00E949F09DD2319F08BE291E008C014
:1015700020919F0533E1239FC0011124825C9E4F7F
:101580000E94CC096CE880E30E949F096FE082E32F
:101590000E949F0962E483E30E949F098091A00555
:1015A00087FF02C064E101C06AE084E30E949F09F2
:1015B0006AE285E30E949F096DE286E30E949F092B
:1015C00064ED87E30E949F0960E088E30E949F0921
:1015D00060E089E30E949F09D11109C0C090810594
:1015E000D0908205E0908305F090840507C0C5E99E
:1015F000CC2EC1ECDC2EED2CCEEDFC2ECAE38F2CD4
:101600009924AA24BB24682D8C2F0E949F09682D41
:1016100085E08C0F0E949F09FE2CED2CDC2CCC2445
:10162000CF5FCE3361F76FEF83E40E949F096FEFC6
:1016300084E40E949F096FEF85E40E949F096FEF89
:1016400086E40E949F09DD2311F066E002C06091EC
:1016500085058DE60E949F0960E089E70E949F0949
:10166000609186058AE70E949F0960E083E70E94F7
:101670009F0960E084E70E949F09D11109C0609131
:101680007D0570917E0580917F059091800504C055
:1016900060EC7AEC89E896E30E940E0ADF91CF9124
:1016A000FF90EF90DF90CF90BF90AF909F908F9082
:1016B000089561E087E00E949F0964E28EE70E943E
:1016C0009F0963E088E00E949F0960E088E00E9433
:1016D0009F0965E087E00E949F0962E085E00E9423
:1016E0009F0983E00E9499098093730584E00E941A
:1016F000990980937205089583E00E949909809367
:10170000730584E00E9499098093720561E087E087
:101710000E949F096AE070E080E090E00E947329D7
:101720000E94590B00000895CF92DF92FF920F9311
:101730001F93CF93DF931F92CDB7DEB7082F162FDD
:101740008EE399830E949F09F02EC02E9981D92E95
:101750008C2D8F19811738F4F60161916F018FE795
:101760000E949F09F5CF64E085E00E949F0983E015
:101770000E9499098093730584E00E9499098093DF
:1017800072050E94502960936E0570936F058093D7
:1017900070059093710569E087E00E949F0981E0E0
:1017A000809375050F90DF91CF911F910F91FF905E
:1017B000DF90CF9008950F931F930E94940B809118
:1017C0007505813099F40E94502900916E051091A1
:1017D0006F052091700530917105601B710B820BB4
:1017E000930B603A76488140910548F380917505E6
:1017F000813031F46EE971E084EE95E00E943C2B7B
:101800001F910F9108950F931F938091750582305A
:1018100021F41092750581E020C08091750581301A
:10182000D9F40E94502900916E0510916F05209106
:10183000700530917105601B710B820B930B613A3F
:1018400076488140910540F061E087E00E949F0961
:101850001092750582E001C080E01F910F910895FC
:10186000CF93DF93EC014AE050E06D2F70E084EEFF
:1018700095E00E940A2C6EE284EE95E00E940E2B09
:10188000BE0184E0769567958A95E1F76F707727BA
:101890004AE050E084EE95E00E940A2C6EE284EE6D
:1018A00095E00E940E2BBE016F7077274AE050E052
:1018B00084EE95E00E940A2CDF91CF910895D82FF5
:1018C000C0E0CD1780F42D9A64E670E080E090E0EF
:1018D0000E9473292D9864E670E080E090E00E94F9
:1018E0007329CF5FEECF6CE271E080E090E00E9460
:1018F0007329E6CF0F931F93CF93DF93EC01062F4D
:1019000015E0115051F0CE010E940531081741F049
:10191000602FCE010E940D31F4CF82E00E945F0C57
:10192000DF91CF911F910F910895A0E0B0E0EBE916
:10193000FCE00C94EB2E482E562EC0E0D0E0612C3B
:10194000712CE12CF12C00E010E041100CC06090F3
:10195000D60586E4689E3001112459E1E52EF12C6C
:101960000CEB15E01EC091E049120FC06090D60547
:10197000E6E46E9E30011124FBE16F0E711C49E21A
:10198000E42EF12C08E715E00CC082E0481209C0F3
:1019900028E1622E77247394EE24E394F12C05ED74
:1019A00015E043018C0E9D1E10927705109276056E
:1019B0003401A62CA818B12CC30101966C01AE14F9
:1019C000BF04A8F4A00EB11E511006C0C3010E94AE
:1019D0000531F501808305C0F5016081C3010E94D6
:1019E0007A0CF50180810E9461063601E2CFC301C5
:1019F000511018C0C3010E940531B82EC6010E94C3
:101A000005312B2D30E0322F2227282B80917605AF
:101A1000909177058217930779F4C0E0D0E05524C0
:101A2000539493CF3601609177050E947A0C6091B0
:101A30007605C6010E947A0CC05EDE4FC13E92E080
:101A4000D90708F482CF852DCDB7DEB7E0E10C943D
:101A5000072F61E082E00E94950C089560E082E02B
:101A60000E94950C8091D505853020F01092D50507
:101A70000E94290D8091D5058093D605089561E0D7
:101A800080E00E94950C61E081E00E94950C089531
:101A900060E080E00E94950C882351F060E081E0D6
:101AA0000E94950C882321F080917805883349F0B5
:101AB0000E94BF060E947A0681E00E94DF060E9413
:101AC0003F0D0895882319F06AEA71E002C06EEABA
:101AD00071E084EE95E00E943C2B0895FF920F93F5
:101AE0001F93CF93DF9369EC7BE084EE95E00E9437
:101AF000E82A40917D0550917E0560917F057091A7
:101B000080052AE030E084EE95E00E94112C63EB22
:101B10007BE084EE95E00E94E82A40918105509197
:101B20008205609183057091840520E130E084EEA8
:101B300095E00E94112C6DE97BE084EE95E00E9417
:101B4000E82A4AE050E06091850584EE95E00E9425
:101B5000392C67E87BE084EE95E00E94E82A4AE0B1
:101B600050E06091860584EE95E00E94392C61E793
:101B70007BE084EE95E00E94E82AC7E8D5E0F12CEE
:101B80008E0188818823A9F0FF2031F061EB71E09C
:101B900084EE95E00E940B2B21964AE050E0F8017C
:101BA000608184EE95E00E94022CF394F8E1FF122C
:101BB000E7CF84EE95E00E94162B6BE57BE084EE88
:101BC00095E00E94E82A4AE050E060919F0584EE8B
:101BD00095E00E94392C66E47BE084EE95E00E945B
:101BE000E82AE091A005E770F0E0EE0FFF1FEE5746
:101BF000FC4F6081718184EE95E00E943C2B61E393
:101C00007BE084EE95E00E94E82A8091A00588712F
:101C1000883069F028F4811113C068E27BE00CC0C1
:101C2000803141F0883161F46CE07BE005C06CE10B
:101C30007BE002C066E17BE084EE95E00E942A2B07
:101C400068EF7AE084EE95E00E94E82A40917905F9
:101C500050917A0560917B0570917C052AE030E017
:101C600084EE95E00E94112C6FED7AE084EE95E011
:101C70000E94E82A8091C10580710E94620D66EC85
:101C80007AE084EE95E00E94E82A8091C105807494
:101C90000E94620D6DEA7AE084EE95E00E94E82AE7
:101CA0008091C10580720E94620D60E97AE084EE45
:101CB00095E00E94E82A88E795E00E94F407AB01CE
:101CC000BC012AE030E084EE95E00E94F32B6BE843
:101CD0007AE084EE95E00E94E82A88E795E00E9489
:101CE000F4079B01AC0160E472E48FE090E00E9495
:101CF000A82EBA01A9012AE030E084EE95E00E9406
:101D0000F32B68E87AE084EE95E00E942A2BCDB7A9
:101D1000DEB7E5E00C94122F8F929F92AF92BF92A4
:101D2000CF92DF92EF92FF92811107C06FE77AE0C6
:101D300084EE95E00E942A2B2FC090E00E94740749
:101D400024E630E040E050E00E94A82ECA01B9012C
:101D50002AE030E040E050E00E94A82E49015A01FC
:101D60006B017C012AE030E0B501A40184EE95E02E
:101D70000E94F32B6EE284EE95E00E940E2B2AE087
:101D800030E0B701A60184EE95E00E94F32B63E7F3
:101D900084EE95E00E944E2BFF90EF90DF90CF9065
:101DA000BF90AF909F908F9008951F93CF93DF9334
:101DB00065E77AE084EE95E00E94E82A8091A1052B
:101DC000813041F46CE57AE084EE95E00E942A2BA4
:101DD00010E050C0823019F465E47AE0F5CF843029
:101DE00019F461E37AE0F0CF853091F766E27AE0AA
:101DF000EBCFC12FD0E0C930D1050CF441C068E36E
:101E0000610F84EE95E00E940E2B6EE17AE084EE85
:101E100095E00E94E82ABE016F5F7F4F4AE050E0E4
:101E200084EE95E00E94D22B63E17AE084EE95E0A7
:101E30000E94E82ACF55DA4FE981E03218F566E0D2
:101E40007AE084EE95E00E94E82A8981803130F0C2
:101E50006DE673E084EE95E00E940B2B69816F7054
:101E600070E06F5F7F4F4AE050E084EE95E00E94A3
:101E7000DB2B1F5F80914A05181708F4BACF0FC0FB
:101E800061E3BECFEF70F0E0EE0FFF1FEE56FC4FA8
:101E90006081718184EE95E00E943C2BEACF6BEE6D
:101EA00079E084EE95E00E94E82A8091B9050E94CD
:101EB0008C0E60ED79E084EE95E00E94E82A809136
:101EC000BA050E948C0E65EB79E084EE95E00E94E5
:101ED000E82A8091BB050E948C0E6AE979E084EEC5
:101EE00095E00E94E82A4091B1055091B2056091B9
:101EF000B3057091B405411551056105710539F1BE
:101F00002AE030E084EE95E00E94112C67E679E04B
:101F100084EE95E00E94E82A8091B5050E94990719
:101F2000AB01BC012AE030E084EE95E00E94112C68
:101F300063E479E084EE95E00E94E82A4AE050E00C
:101F40006091B60584EE95E00E94392C06C06AE3E4
:101F500079E084EE95E00E942A2B6DE179E084EE31
:101F600095E00E94E82A6091B7057091B8054AE0B3
:101F700050E084EE95E00E94232C60E079E084EE4E
:101F800095E00E94E82A6091B005603450F470E05A
:101F90006F5F7F4F4AE050E084EE95E00E94DB2BBC
:101FA00006C067EF78E084EE95E00E942A2B6AED88
:101FB00078E084EE95E00E94E82A8091AF0580FFEA
:101FC00003C063EB71E002C067EB71E084EE95E063
:101FD0000E943C2B6DEB78E084EE95E00E94E82AAD
:101FE0008091AF0582700E94620D6EE978E084EE08
:101FF00095E00E94E82A8091AF0584700E94620DEE
:102000006FE778E084EE95E00E94E82A8091AF05C2
:1020100088700E94620DDF91CF911F9108950F93F8
:102020001F93CF93DF93209147052F3FA9F56FEFC3
:1020300075E084EE95E00E94E82A88E893E00E942B
:10204000300C6EED75E084EE95E00E94E82A8091F8
:102050004805909149050E94300C6BEA75E084EECA
:1020600095E00E942A2B68E875E084EE95E00E94D6
:102070002A2B60E775E084EE95E00E942A2B6BE442
:1020800075E084EE95E00E942A2B84EE95E00E9494
:10209000162B0E94D50E68C012160CF065C03327AF
:1020A00027FD309580914A0590E0821793070CF444
:1020B0005BC066E375E084EE95E00E94E82A6091DB
:1020C0004705772767FD70954AE050E084EE95E07C
:1020D0000E94DB2B6BE075E084EE95E00E94E82A1D
:1020E00010E008E280914B051817D0F5C12FD0E021
:1020F000CC0FDD1FC45BDA4F288130E080914705AB
:10210000992787FD909501972817390739F56BEBCB
:1021100071E084EE95E00E940B2B4AE050E0602FC6
:1021200084EE95E00E94022C6FEB71E084EE95E066
:102130000E940B2BE981EF70F0E0EE0FFF1FEE56CF
:10214000FC4F6081718184EE95E00E940B2B63EC63
:1021500071E084EE95E00E940B2B0F5F1F5FC2CFF2
:1021600084EE95E00E94162BDF91CF911F910F9185
:102170000895FF920F931F93CF93DF93C7E8D5E0A5
:10218000F12C8E0188818823D1F165EC71E084EE19
:1021900095E00E940B2B4AE050E06F2D84EE95E015
:1021A0000E94022C62ED71E084EE95E00E940B2B00
:1021B0002196F801208130E0A0E1B7E20E94622E72
:1021C0009B01AC01A0918605B0E00E94712EAB018D
:1021D000BC0180917D0590917E05A0917F05B09115
:1021E0008005480F591F6A1F7B1F2AE030E084EEEC
:1021F00095E00E94112CF394F8E1FF12C2CFCDB705
:10220000DEB7E5E00C94122F1092E10485E6E2EED1
:10221000F4E0DF011D928A95E9F70895CF93C82F66
:102220008F3719F0883009F045C0E091E104EE23C2
:10223000D9F1E150E093E104F0E0EE51FB4F108260
:102240006DE070E084EE95E00E945906C0E0809158
:10225000E104C81760F4EC2FF0E0EE51FB4F608111
:1022600070E084EE95E00E945906CF5FF0CF60E207
:1022700070E084EE95E00E9459066DE070E084EE17
:1022800095E00E945906C0E08091E104C81778F5F6
:10229000EC2FF0E0EE51FB4F608170E084EE95E0B2
:1022A0000E945906CF5FF0CF67E084EE95E00E9470
:1022B0000E2B1DC08B3119F40E9404111AC08D30F1
:1022C000C1F08A30B1F08091E104843668F76C2F58
:1022D00070E084EE95E00E945906E091E10481E00F
:1022E0008E0F8093E104F0E0EE51FB4FC08380E05D
:1022F00001C081E0CF910895CF93C82F0E9450294B
:102300006093CA047093CB048093CC049093CD0463
:10231000C093DF04CC2329F040E051EE60E070E090
:1023200004C040E855E260E070E084EE95E00E9471
:10233000982DCF9108959091CE04492F4F7050E081
:10234000BA016F5F7F4F292F30E0E4E03595279584
:10235000EA95E1F76217730759F0FA01E153FB4F71
:10236000808381E0890F8F70907F892B8093CE04CA
:1023700008956EE770E084EE95E00E945906089596
:10238000A3E1B1E0E6ECF1E10C94EC2EE7E8F5E036
:10239000712C8191882321F0739428E17212F9CF76
:1023A00066ED71E084EE95E00E943C2B4AE050E03F
:1023B000672D84EE95E00E94392C80E00E947E0A11
:1023C0000E94590B8E010E5F1F4FC12CD12C76013C
:1023D000C39466246A945C2C0E9444294B015C01DE
:1023E0002091860530E0A0E1B7E20E94622E9B01B9
:1023F000AC01C701B6010E94842E20917D05309169
:102400007E0540917F0550918005620F731F841FE8
:10241000951F2091BD053091BE054091BF0550919B
:10242000C005261737074807590718F4F8016082D6
:1024300025C08C2D0E94B20961E070E080E090E040
:102440000E947329F80110820E94442968197909B1
:102450008A099B09643F71408105910540F40E94FF
:10246000C809F8019081981778F78083EDCF50FE66
:1024700003C02C982D9A02C02C9A2D982FEFC21AC7
:10248000D20AE20AF20A0F5F1F4F8FEFC816D1047B
:10249000E104F10409F09FCFCE019395FC01D82E01
:1024A0007FEF68EC2E2F281B271510F051E056C047
:1024B000DE01129651E02FEF41E03D91321710F00E
:1024C000322F01C0452F5F5F5F3F11F0232FF5CF03
:1024D0004193242F30E0A1E0B0E0AC0FBD1FA20F6C
:1024E000B31F5C93413079F0DE01A20FB31F5C9300
:1024F000423049F0AFEFBFEFAC0FBD1FA20FB31FCB
:102500006C934E3F78F6A2E0B0E0AC0FBD1FA20F77
:10251000B31F7C934D3F30F6A3E0B0E0AC0FBD1F7E
:10252000A20FB31F6C93BECF452F242F30E0FC01C8
:10253000E20FF31F6081AFEFB0E0AC0FBD1FA20F41
:10254000B31F2C91621748F44150DC01A40FB11D58
:102550002C9120836C934111E8CF5F5F571520F3D6
:10256000372D369520E0231770F4DC01A20FB11D42
:102570004C91522F530FFC01E50FF11D50815C93DC
:1025800040832E5FF0CFF7E8EF2EF5E0FF2E8C01B1
:10259000802F8D19871598F4F801C1908F014AE0BA
:1025A00050E06C2D84EE95E00E94022C6CE284EEEB
:1025B00095E00E940E2BF701C1927F01E9CF84EED6
:1025C00095E00E94162B81E0CD5EDE4FEFE00C948B
:1025D000082F1F920F920FB60F9211240F931F9383
:1025E0002F933F934F935F936F937F938F939F931B
:1025F000AF93BF93EF93FF934091C1055091C205F4
:102600006091C3057091C40589B18A019B01007472
:1026100011272227332783FB882780F990E0A0E049
:10262000B0E0081719072A073B0709F468C0809132
:102630008400909185001092850010928400209172
:10264000A70421115CC045FD02C096958795853C85
:1026500029E09207C0F180910A0190E0A0E0B0E08B
:102660000CE176956795579547950A95D1F74115F1
:1026700051056105710521F441E050E060E070E032
:10268000481759076A077B07D8F480910A018F3FE2
:10269000B9F040E080910A01481780F4842F90E05F
:1026A000880F991FFC01E957FB4F20813181FC0104
:1026B000E55FFE4F318320834F5FECCF1092A8047B
:1026C00010920A011CC08D3B22E09207A8F02091D5
:1026D0000A01203188F410910A0121E0210F209392
:1026E0000A010E94DE08E12FF0E0EE0FFF1FE9571C
:1026F000FB4F9183808303C08FEF80930A01FF918A
:10270000EF91BF91AF919F918F917F916F915F9169
:102710004F913F912F911F910F910F900FBE0F90EE
:102720001F90189583E0809380008AE18093810058
:102730008FEF9FEF909389008093880010926F0035
:1027400088E080936D00E8E6F0E08081846080831B
:102750000895CF93DF930E942E0D8091D60584308B
:1027600039F585E00E94692AC1E0D0E0892B11F497
:10277000C0E0D0E086E00E94692A892B19F082E04F
:1027800090E002C080E090E08C2B9D2B8230910580
:1027900039F08330910539F0019739F481E006C0B2
:1027A0001092D60505C082E001C083E08093D60573
:1027B000DF91CF9108956F3018F086958058089575
:1027C00089E0689F802D11240895A0E0B0E0EBEE31
:1027D000F3E10C94F32EC82F0E9450290091380485
:1027E0001091390420913A0430913B046B017C0133
:1027F000C01AD10AE20AF30A9701860149E8C41611
:1028000043E1D406E104F10410F010923C0460931B
:1028100038047093390480933A0490933B042091D8
:10282000A7048FEF820F8230E8F5E0913C04EE239D
:1028300009F46EC1E13011F482E0D8C1E03178F5DD
:1028400081E08E0F80933C04F0E0E957FB4FC0839A
:10285000803109F0D4C1E9E8F4E0213029F4A18104
:10286000A695A695808108C080819181A92FA69503
:10287000A695A69596958795A03148F4B0E090E08E
:10288000AA0FBB1FA55FBE4F11969C938E9310920B
:10289000A804329684E0E739F807F9F6B0C110923F
:1028A0003C04ADC1233009F023C1E0913C04E111A7
:1028B00018C0CF3009F011C10E9444290091B5041D
:1028C0001091B6042091B7043091B804601B710BCD
:1028D000820B930B623071058105910508F089C167
:1028E000FCC0E73148F481E08E0F80933C04F0E0B7
:1028F000EA57FB4FC083F1C0E73109F0ECC0C111CA
:10290000EAC040E050E0ABE0CA01B3E0880F991F95
:10291000BA95E1F7A49F9001A59F300D1124F9010C
:10292000E957FB4F6081E1817E2F77707595679540
:10293000FC01EE0FFF1FE55FFE4F71836083F9011D
:10294000E857FB4FB081B695B695B695E181FE2F5D
:10295000F295FF0FF07E6F2F6B2BE695E695E695CF
:102960007E2F777075956795FC01EE0FFF1FE35F73
:10297000FE4F71836083F901E757FB4FB081B29539
:10298000B695B695B370C181DC2FDD0FDD0F6D2FCD
:102990006B2BC295C695C695C370E281E170EE0FB0
:1029A000EE0F7E2F7C2B75956795FC01EE0FFF1FB8
:1029B000E15FFE4F71836083F901E557FB4FB08102
:1029C000B695E181FE2FF795FF27F7956F2F6B2BBB
:1029D000E6957E2F777075956795FC01EE0FFF1FCA
:1029E000EF5EFE4F71836083F901E457FB4FB081C6
:1029F000B295BF70E181FE2FF295F07F6F2F6B2BA8
:102A0000E295EF707E2F777075956795FC01EE0F5C
:102A1000FF1FED5EFE4F71836083F901E357FB4FAB
:102A2000B081BB1FBB27BB1FC181DC2FDD0F6D2F0A
:102A30006B2BCC1FCC27CC1FE281E370EE0F7E2FD7
:102A40007C2B75956795FC01EE0FFF1FEB5EFE4F2B
:102A500071836083F901E157FB4FB081B695B6955C
:102A6000E181FE2FF295FF0FFF0FF07C6F2F6B2B94
:102A7000E695E6957E2F777075956795FC01EE0FCC
:102A8000FF1FE95EFE4F71836083F901E057FB4F42
:102A900020812295269527703181E32FEE0FEE0FCE
:102AA000EE0F6E2F622B732F72957695777075955A
:102AB0006795FC01EE0FFF1FE75EFE4F7183608399
:102AC0004F5F5F4F4230510509F01ECF80919D044A
:102AD00083FF1092A80410923C040E944429609342
:102AE000B5047093B6048093B7049093B80487C07C
:102AF000243009F084C060913C0461110BC0C83AD5
:102B0000B1F4109277051092760588EA0E9461066A
:102B100081E06CC0613019F4C093370404C06230A6
:102B200031F4C09336048C2F0E9461065AC0E091A4
:102B300036042E2F30E0220F331F462F50E0C901FC
:102B40000296841795073CF0633268F7FA01EC5758
:102B5000FB4FC083E8CF2D5F3F4F8C2F90E06091FB
:102B60007605709177054217530749F4982F882707
:102B700086279727909377058093760532C068174C
:102B8000790769F580913704813049F5E13118F012
:102B900080E180933604F0903604C8E8D4E000E089
:102BA00010E00F15D0F4FE013197808190E0982F4E
:102BB00088272881822B43E0969587954A95E1F7EF
:102BC0000E94DE08F801EE0FFF1FE55FFE4F9183C4
:102BD00080830F5F1F4F2296E4CF1092A8041092BB
:102BE0003C0480913C04882351F08F5F80933C0427
:102BF00006C080913C048F5F80933C046ECFCDB7BC
:102C0000DEB7E8E00C940F2FCF93DF93E82FF0E0CE
:102C1000E454FA4FE185E03150F4F894F0E0EE0F1F
:102C2000FF1FE55FFE4F8081918178945DC08EE04B
:102C30008E0F8B3058F4F0E0E25FF10924E62E9F0E
:102C4000C0012F9F900D11240C964EC0E03F09F457
:102C500046C038F4E13181F0E23191F0E03139F4ED
:102C600009C0ED3FB1F1EE3FB9F1E13F79F180E00C
:102C700092E03AC082E101C083E10E94922A34C00E
:102C800085E00E94692AC1E0D0E0892B11F4C0E000
:102C9000D0E086E00E94692A892B19F082E090E05A
:102CA00002C080E090E08C2B9D2B8230910541F09A
:102CB0008330910541F00197A9F086EA92E014C0B3
:102CC0008CE090E011C089E591E00EC086E090E0D4
:102CD0000BC08AEF93E008C08FEF93E005C080E05F
:102CE00090E002C084EF93E0DF91CF910895A2E2DB
:102CF000B0E0EDE7F6E10C94E92E9E012F5F3F4F27
:102D000080E1D9011D928A95E9F764E072E084EED2
:102D100095E029A33AA30E943C2B0E947C0B1D8ABC
:102D20001E8A1F8A188E312C212C00E0812C912CB8
:102D3000540170EC472E7DE9572E78E5672E75E338
:102D4000772EE0E5CE2EE3ECDE2EE12CF12C84EFA5
:102D500091E0A0E0B0E08D8F9E8FAF8FB8A380ECA4
:102D600097EFAAEBB7E3898F9A8FAB8FBC8F80EC7C
:102D70009DE9A8E5B5E3898B9A8BAB8BBC8B84EE80
:102D800095E00E94502C892B09F4E1C084EE95E077
:102D90000E947D2C9C0133272C32310509F442C05E
:102DA000ACF42332310509F0ABC019821A821B82C0
:102DB0001C821D821E821F82188619861A861B8617
:102DC0001C861D861E861F86188A60C02434310525
:102DD00029F02335310509F4B2C092C064E484EED1
:102DE00095E00E940E2B2AE030E040EC5DE968E5BA
:102DF00075E384EE95E00E949C2B6CE284EE95E0F6
:102E00000E940E2B2AE030E040EC57EF6AEB77E3AC
:102E100084EE95E00E949C2B6CE284EE95E00E948B
:102E20004E2BADCF0F5F043009F0A9CF29813A8135
:102E30004B815C81A8EEB3E00E94712E698B7A8B86
:102E40008B8B9C8B2D813E814F8158850E94712EEA
:102E5000698F7A8F8B8F9C8F29853A854B855C850E
:102E60002D8F3E8F4F8F58A32D853E854F855889D6
:102E70000E94712E6B017C0160323EE47307810574
:102E8000910530F462E38CE10E949F0900E077CF66
:102E9000603345E774078105910510F462E2F3CFD2
:102EA00060345CE975078105910510F466E2EBCFAB
:102EB00080E5C81683ECD806E104F10410F462E161
:102EC000E2CF90E6C9169AEED906E104F10410F4B7
:102ED00065E1D9CFA0E7CA16A1E1DA06A1E0EA06CA
:102EE000F10410F461E0CFCFB0EACB16B6E8DB0610
:102EF000B1E0EB06F10410F463E0C5CF65E0C3CFA9
:102F000010ED180F1A3008F03ACFE1E0F0E0EC0FC6
:102F1000FD1F24E0029FE00DF11D1124208131816D
:102F200042815381AAE0B0E00E94712E610F711DB1
:102F3000811D911D608371838283938320CF498893
:102F40005A886B887C88812C912C540118CF81146D
:102F50009104A104B10489F4C301B2010E940E0AD4
:102F600061E070E080E090E00E9473291D8A1E8A73
:102F70001F8A188E312C22242A948D8D9E8DAF8D20
:102F8000B8A188169906AA06BB06D0F40E94C80903
:102F90002D893E894F89588D280F311D411D511DA6
:102FA0002D8B3E8B4F8B588F381608F4382E821598
:102FB00008F4282E3FEF831A930AA30AB30A56C0D7
:102FC000C301B20128EE33E040E050E00E94A82E99
:102FD000BA01A9012AE030E084EE95E00E94F32BCB
:102FE0006CE284EE95E00E940E2B4AE050E0632DE7
:102FF00084EE95E00E94022C6CE284EE95E00E9443
:103000000E2B6D897E898F89988DA50194010E9470
:10301000A82EBA01A9012AE030E084EE95E00E94D2
:10302000F32B6CE284EE95E00E940E2B4AE050E018
:10303000622D84EE95E00E94022C6CE284EE95E015
:103040000E944E2B4C0C5D1C6E1C7F1C898D9A8D32
:10305000AB8DBC8D84159505A605B70520F4498870
:103060005A886B887C88812C912C540129893A8953
:103070004B895C89283E33404105510509F07FCEDC
:10308000A296E2E10C94052FACE1B0E0EAE4F8E1AD
:103090000C94F32E0E9450296B017C0181E00E9468
:1030A0007E0A14E703E0198361E0CE0101960E94D5
:1030B000DB0B009375050E94590B6AEF70E080E00E
:1030C00090E00E94732980917505833089F484EE25
:1030D00095E00E94502C892B59F40E9450296C19BC
:1030E0007D098E099F096038734C894C9140D8F254
:1030F00080917505833009F44FC08FE70E947709EE
:103100000E948A098983843511F083E05CC00E94A3
:103110008A0910924805809349050E948A092091E6
:10312000480530914905280F311D309349052093FA
:1031300048050E948A0980934A050E948A09809363
:103140004B05813110F7F12C0F2D10E080914B05CC
:1031500090E0880F991F0817190740F40E948A0908
:10316000F801E45BFA4F8083F394EECF80E7898324
:1031700061E0CE0101960E94DB0B83E08093750530
:103180000E94590B62E370E080E090E00E94732996
:1031900080917505833011F482E015C08FE70E949D
:1031A00077090E948A098983803509F0AECF01EA48
:1031B00015E00E948A09F80181938F01F5E00C3B2C
:1031C0001F07B9F781E06C96E8E00C940F2F80910F
:1031D0004705992787FD9095A92FB92FFC013196B6
:1031E000EB30F10508F066C0EC5CFF4F0C94202F2B
:1031F00062E778E084EE95E00E942A2B88E893E06D
:103200000E94300C6AE578E084EE95E00E942A2B5B
:1032100065E378E084EE95E00E942A2B6BE078E08D
:1032200084EE95E00E942A2B6AEE77E084EE95E02A
:103230000E942A2B6DEB77E084EE95E00E942A2B0A
:1032400067E977E084EE95E00E942A2B63E777E058
:1032500084EE95E00E942A2B6CE477E084EE95E002
:103260000E942A2B84EE95E00E94162B0E946E0D80
:1032700021C06FE277E01AC06AE077E017C065EF1F
:1032800076E014C066ED76E011C062E976E00EC02B
:103290006DE776E00BC068E676E084EE95E00E948C
:1032A0002A2B62E276E002C06CE076E084EE95E0E4
:1032B0000E942A2B6AE070E080E090E00E9473296F
:1032C00084EE95E00E94502C892B29F084EE95E045
:1032D0000E947D2CF5CF0895ACE1B0E0E2E7F9E182
:1032E0000C94F32E909147059F3F09F023C1482F7E
:1032F00050E0FA013A97EF36F10508F00FC1E15CB2
:10330000FF4F0C94202F61E172E0A0C06DE172E0EC
:1033100084EE95E00E943C2B85E789838BE1E1EA0E
:10332000F5E0DE01129601900D928A95E1F76CE1CD
:10333000CE0101960E94DB0B0E94590B83E0809323
:10334000750568EC70E080E090E00E947329809140
:103350007505843009F0E2C08FE70E9477090E946A
:103360008A098983853509F0D9C06DEE74E084EE51
:1033700095E00E942A2B6FEC74E084EE95E00E94A9
:103380002A2B61EB74E096C065E372E084EE95E071
:103390000E943C2B89E6898361E0CE0101960E9460
:1033A000DB0B0E94590B83E08093750568EC70E09D
:1033B00080E090E00E94732980917505843009F0C7
:1033C000ADC08FE70E9477090E948A0989838E0128
:1033D0000E5F1F4F7E014DE1E40EF11C0E948A0931
:1033E000F80181938F01EE15FF05C1F78BE1FE0116
:1033F0003296A1EAB5E001900D928A95E1F78981B4
:10340000893409F08BC063E974E084EE95E00E9492
:103410002A2B65E774E084EE95E00E942A2B67E58D
:1034200074E048C06FE472E084EE95E00E943C2BAB
:103430008EEF8093470572C08052875080539091E1
:103440004A05981708F066C06EE572E084EE95E0D4
:103450000E943C2B63C084E18093470560E274E0E6
:1034600029C085E18093470569EE73E023C086E1BA
:103470008093470562EB73E01DC087E180934705A9
:1034800068E673E017C088E18093470567E573E05D
:1034900011C089E18093470563E473E00BC08AE1C2
:1034A000809347056EE273E005C08BE1809347058A
:1034B00066E073E084EE95E00E942A2B2FC06CEE4C
:1034C00072E084EE95E00E942A2B8091AF0591E096
:1034D0001DC066ED72E084EE95E00E942A2B80917B
:1034E000AF0592E013C061EC72E084EE95E00E94BB
:1034F0002A2B8091AF0594E009C066EA72E084EE61
:1035000095E00E942A2B8091AF0598E0892780934F
:10351000AF058FEF809347050E940F1084EE95E072
:103520000E94502C892B09F45BC184EE95E00E9427
:103530007D2CF4CF0E940E11882309F451C1809193
:10354000E104811104C08FEF8093470541C140E041
:1035500050E060E070E082EE94E00E94972F40918E
:103560004705042F112707FD1095212F312FF80152
:103570003197EB31F10508F01BC1E255FF4F0C9478
:10358000202F552747FD509520914A0530E02417FC
:1035900035070CF40DC18B019C0101501109210963
:1035A0003109003211052105310558F0C0904B0555
:1035B000EDE4F5E0F12CD12CA8E2EA2E41505109BE
:1035C0000FC0FA01EF55FA4F61506083D9C0DF0197
:1035D00011972C9130E02417350729F0F394329697
:1035E000FC10F5CFCBC00E2D10E020E030E0061728
:1035F00017072807390741F42081DA01AF55BA4F80
:1036000011962C93DD24D394E394E8CF6F3F71059A
:103610008105910511F008F0CBC06093B905B0C0E9
:103620006F3F71058105910511F008F0C1C06093ED
:10363000BA05A6C06F3F71058105910511F008F02C
:10364000B7C06093BB059CC02091E2042062203784
:10365000E9F440E050E060E070E083EE94E00E9426
:10366000972F9B01AC01DC01CB010197A109B109A6
:103670000897A105B10508F0AEC0A4EDB0E30E9423
:10368000712E6A5E7C4A8A46954E24C02636E9F43D
:1036900040E050E060E070E083EE94E00E94972FFD
:1036A0009B01AC01DC01CB010197A109B10907978E
:1036B000A105B10508F08FC0A8EAB1E60E94712EFD
:1036C000645E7C438E46944E05C06115710581058C
:1036D000910579F08B019C01005C1D49284535431B
:1036E0000130FAE51F07F2E62F07F2E03F0708F086
:1036F0005FC06093B1057093B2058093B30590935A
:10370000B4053EC06F3F71058105910511F008F0C9
:103710004FC06093B50534C08B019C010150110965
:10372000210931090F3F11052105310508F040C07D
:103730006093B60525C08B019C01045C19402109EA
:1037400031090D344DE114072105310528F470933A
:10375000B8056093B70514C0611571058105910521
:1037600021F48FEF8093B0050BC0613471058105A2
:103770009105F0F461506093B00502C0DD20C1F006
:103780008091E00481111AC0809181059091820599
:10379000A0918305B09184050196A11DB11D809370
:1037A000810590938205A0938305B093840506C09C
:1037B00060E772E084EE95E00E943C2B0E940411C9
:1037C0008FEF809347056AE084EE95E00E944E2BD0
:1037D0000E940F1005C061E070E080E090E07ACFB9
:1037E0006C96E8E00C940F2F6AE572E084EE95E0A9
:1037F0000E942A2B62E472E084EE95E00E942A2B5C
:1038000084EE95E00E94502C892B31F084EE95E0F7
:103810000E947D2C0E946C190E944418823029F06D
:10382000833051F46DE072E002C064E272E084EE35
:1038300095E00E942A2B08958FEF80934705109200
:10384000E0040E940F10809147058E3F69F084EEDE
:1038500095E00E94502C892BB1F384EE95E00E94F4
:103860007D2C0E946C19EFCF08950F931F93109138
:1038700047051F3F09F0D2C0893409F457C000F54D
:10388000883309F469C058F4803309F477C008F02C
:1038900061C08B3109F440C08132B1F1B9C08134CB
:1038A00009F487C030F4893309F466C0803461F1CB
:1038B000AFC0823409F48EC0863409F448C0A8C071
:1038C000823609F487C078F4883531F128F48235DE
:1038D000C1F18335E1F09CC08A3509F494C081368A
:1038E00009F467C095C0823761F128F4863679F112
:1038F0008936E1F08DC0883779F08A3709F483C0C2
:10390000833709F085C003C061E172E015C00E94F1
:103910003F0D6EE872E004C00E94480D68EA72E054
:1039200084EE95E00E943C2B8EEF70C00E947A06D8
:103930000E94BF0667EC72E084EE95E00E943C2B8B
:1039400067C081E00E94DF0660EE72E0F5CF0E9462
:10395000B9105EC080535AC06AEF71E084EE95E002
:103960000E942A2B9091A00588E0890F8871977E8C
:10397000892B8093A0051AC089E048C067EE71E0EA
:1039800084EE95E00E942A2B8091C1059091C2059A
:10399000A091C305B091C40520E182278093C105A1
:1039A0009093C205A093C305B093C4051093470537
:1039B0002FC061ED71E084EE95E00E942A2B80918A
:1039C000C1059091C205A091C305B091C40540E422
:1039D000842710C060EC71E084EE95E00E942A2BF1
:1039E0008091C1059091C205A091C305B091C40515
:1039F00020E282278093C1059093C205A093C3055E
:103A0000B093C40502C00E94F41B8FEF809347055A
:103A1000809147058E3F09F0D4C0DDC00E940E1191
:103A2000882309F4D8C08091E104811104C08FEF8C
:103A300080934705C6C040E050E060E070E082EE51
:103A400094E00E94972F00914705112707FD1095DC
:103A5000212F312FF8013197E930F10508F0B4C07A
:103A6000E753FF4F0C94202F8B019C01015C1D49F3
:103A7000284535430F3F19452246324008F0A4C07F
:103A800060937D0570937E0580937F0590938005FC
:103A900077C060938105709382058093830590932E
:103AA000840581E08093E0046BC068307105810576
:103AB000910508F089C06093850562C08B019C0167
:103AC00001501109210931090A301105210531057B
:103AD00008F07AC06093860553C061EB71E082EE16
:103AE00094E00E94D13010E0009799F00E94AB3032
:103AF000009779F0183130F4E12FF0E0E858FA4FF0
:103B000087871F5F61EB71E080E090E00E94D13019
:103B1000EBCF1831A8F5E12FF0E0E858FA4F1786FF
:103B20001F5FF7CF653071058105910508F04CC026
:103B300060939F0525C08B019C010150110921094B
:103B400031090630110521053105F0F52091A00558
:103B5000287F262B2093A00513C08B019C010150C8
:103B60001109210931090115124C2140310560F577
:103B70006093790570937A0580937B0590937C051B
:103B80008091E004811113C080918105909182059C
:103B9000A0918305B09184050196A11DB11D80936C
:103BA000810590938205A0938305B09384050E94BC
:103BB00004118FEF809347056AE084EE95E00E9440
:103BC0004E2B0E94E71807C060E772E084EE95E094
:103BD0000E943C2BECCF1F910F9108958FEF8093A3
:103BE00047051092E0040E94E718809147058E3F38
:103BF00069F084EE95E00E94502C892BB1F384EE9D
:103C000095E00E947D2C0E94351CEFCF6AE070E0A9
:103C100080E090E00E94732984EE95E00E94502C91
:103C2000892B29F084EE95E00E947D2CF5CF089534
:103C3000CF93C82F682F84EE95E00E94AA2C909114
:103C40006C059C2790936C05CF910895A1E0B0E09E
:103C5000ECE2FEE10C94F92E99830E94181E9981E2
:103C6000892F0E94181E2196E2E00C94152F1F93B5
:103C7000CF93DF93182FEB0110926C0565EB70E08A
:103C800084EE95E00E94590662E670E084EE95E0CD
:103C90000E945906812F0E94181ECE010E94261EE6
:103CA000DF91CF911F91089560916C0584EE95E0AE
:103CB0000E94AA2C0895A1E2B0E0E1E6FEE10C9496
:103CC000F52E7B018A018C3009F453C108F040C005
:103CD000863009F4BCC018F5833009F491C070F443
:103CE000813009F472C0823009F04AC26BE170E0A1
:103CF00082E00E94371E01EA15E078C0843009F4A2
:103D000087C0853009F03CC260914B0570E0660FBA
:103D1000771F85E00E94371E0CE415E086C08930CD
:103D200009F4A7C070F4873009F49BC0883009F00B
:103D300027C261E070E088E00E94371E8091D605BE
:103D400025C28A3009F4CAC08B3009F4F2C018C207
:103D50008A3609F475C1D8F4873609F43AC138F4C3
:103D6000853609F40EC1863609F41FC109C28836AA
:103D700009F437C1893609F003C261E070E089E6D1
:103D80000E94371E0E947A060E94BF06F7C18D3638
:103D900009F4D4C138F48B3609F491C18C3609F496
:103DA0009AC1EEC18E3609F4DEC1873C09F0E8C144
:103DB00061E070E087EC0E94371E81E00E94181ECF
:103DC0000E94541E10926D05E5C169E270E081E029
:103DD0000E94371E08E715E0F80181918F010E94CB
:103DE000181EF5E0013A1F07B9F7D2C1F801819119
:103DF0008F010E94181EF5E00C3B1F07B9F7C8C1E0
:103E000061E070E083E00E94371E0E944418BEC14A
:103E100061E070E084E00E94371E81E00E94181E7D
:103E20000E94541E0E947716B5C180914B0590E008
:103E3000880F991F98012C5435402817390708F02E
:103E4000A7C1F80181918F010E94181EEECF62E098
:103E500070E086E00E94371E88E893E00E94261EEC
:103E600097C161E070E087E00E94371E80914A05AB
:103E70008DC186E6898361E0CE0101960E94DB0B4D
:103E80000E94590B83E08093750568EC70E080E038
:103E900090E00E947329809175058430D9F48FE7F2
:103EA0000E9477090E948A098983863469F460E256
:103EB00070E089E00E94371E10E20E948A090E9489
:103EC000181E1150D1F764C161E070E089E00E94D2
:103ED000371E54C161E070E089E055C169E170E0CE
:103EE0008AE00E94371E82E08093BC052091740511
:103EF0008091C1059091C205A091C305B091C40500
:103F0000222311F0806801C08F778093C1059093C0
:103F1000C205A093C305B093C4050CEB15E0F801EE
:103F200081918F010E94181EF5E0053D1F07B9F72A
:103F30002FC161E270E08BE00E94371E8091A804DF
:103F40008F3F39F08091A80491E0980F9093A804D6
:103F500002C08091A8040E94181E10E0812F0E94C8
:103F600004160E9409090E94261E1F5F1031B1F736
:103F70000FC161E070E08CE00E94371E8091D50592
:103F800005C161E070E085E60E94371E89E2E8160F
:103F9000F10409F0FAC0D801E8E7F5E08D918193CA
:103FA00085E0E13AF807D1F7E9C061E070E086E624
:103FB0000E94371EEBE1EE16F10409F0E6C0D801CD
:103FC000E1EAF5E08D91819385E0EC3BF807D1F7CC
:103FD000D5C061E070E087E60E94371E0E943F0D69
:103FE000CDC061E070E088E60E94371E85E78983D6
:103FF0008BE1E1EAF5E0DE01129601900D928A95DF
:10400000E1F76CE1CE0101960E94DB0B0E94590B97
:1040100083E08093750560E273E080E090E00E94A9
:10402000732980917505843009F0AFC08FE70E9435
:1040300077090E948A098983853509F0A6C09EC048
:1040400061E070E08AE60E94371E89E6898361E0BC
:10405000CE0101960E94DB0B0E94590B83E08093F6
:10406000750560E273E080E090E00E947329809122
:104070007505843009F089C08FE70E9477090E9496
:104080008A0989838E010E5F1F4F7E01EDE1EE0EDE
:10409000F11C0E948A09F80181938F01EE15FF053A
:1040A000C1F78BE1FE013296A1EAB5E001900D92D5
:1040B0008A95E1F78981893409F067C05FC061E0C2
:1040C00070E08BE60E94371EF80180818093D60550
:1040D0000E94480D53C061E070E08CE60E94371EDC
:1040E000F0E2EF16F10461F487E6898380E2F801DB
:1040F000DE01129601900D928A95E1F761E203C00C
:1041000087E4898361E0CE0101960E94DB0B0E9467
:10411000590B83E0809375056CE474E080E090E0D7
:104120000E94732980917505843079F58FE70E948C
:1041300077090E948A09873441F520C061E070E068
:104140008DE60E94371E89E1E816F104F1F4D801EA
:10415000ECEBF5E08D91819385E0E53DF807D1F733
:104160000E9492130BC061E070E08EE60E94371E41
:10417000F80180818093D5050E94290D81E006C059
:1041800061E070E08AEC0E94371E80E00E94181EF9
:104190000E94541EA196E6E00C94112FA0E0B0E01E
:1041A000E4EDF0E20C94F32ECAECD3E014E606E062
:1041B00035E0F32E44E0E42E53E0D52E62E0C62E27
:1041C00084EE95E00E94502C892B09F49BC084EE6C
:1041D00095E00E947D2C282F809335044091340473
:1041E00050E04730510560F7FA01EE52FF4F0C9452
:1041F000202F853B29F781E080933404E1CF82367C
:1042000009F07DC0C0923404DBCF809333048093E7
:104210003204D0923404D4CF9C013327309331043C
:104220002093300490913204982790933204E092C6
:104230003404C6CF382F22274091300450913104E6
:10424000242B352B30933104209330049091320489
:10425000982790933204F09234042536310508F4FF
:10426000AFCF61E070E08CEC0E94371E81E00E94CD
:10427000181E0E94541E43C020912E0430912F041A
:10428000F901E653FC4F8083909132049827909374
:104290003204C901019690932F0480932E0420913B
:1042A0003004309131048217930708F489CF0093CA
:1042B000340486CF8091320482130BC060912E04A7
:1042C00070912F044AEC53E0809133040E945B1EEE
:1042D0000DC062E070E08BEC0E94371E80913304C9
:1042E0000E94181E80916C050E94181EFE01812FED
:1042F00011928A95E9F710922F0410922E041092D1
:1043000034045ECFCDB7DEB7E8E00C940F2F81E028
:1043100080936D0580916D05882349F084EE95E0CA
:104320000E94502C892BB1F30E94CE20F3CF089528
:10433000AAE2B0E0EEE9F1E20C94F12E0E944429E9
:104340006B017C0181E00E947E0A84EE95E00E9470
:10435000502C892B29F084EE95E00E947D2CF5CF1E
:104360002D9811E072E6B72EE9E2AE2E03E00E942E
:1043700044296C197D098E099F09693C71058105E5
:104380009105D0F11123C1F10E9444296B017C01F8
:104390002C9A80ED97E00E94A807B982E8E7F5E043
:1043A000DE0112968A2D01900D928A95E1F76AE25C
:1043B000CE0101960E94DB0B2C9880E090E00E94D9
:1043C000A807009375050E94590B62E370E080E036
:1043D00090E00E94732980917505843061F4009308
:1043E00075058FE70E9477090E948A0911E08234DF
:1043F00019F410E001C011E08BE00E94692A892BBA
:1044000081F411E00EC02D9A2C9A84EE95E00E9462
:104410007D2C8D309105A9F05CF40A9791F02D98D0
:104420002C9884EE95E00E94502C892B61F79FCF49
:104430008332910579F08234910589F70E948721B2
:10444000EECF62EB71E084EE95E00E942A2B0E9491
:10445000EE1DE5CF0E947716E2CF8F929F92AF922A
:10446000BF92CF92DF92EF92FF921F93CF93DF9391
:104470008BE00E94692A892B09F089C068EC70E002
:1044800080E090E00E94732980E090E00E94A807FD
:104490000E9444294B015C016B017C0180ECC80E39
:1044A00082E1D81EE11CF11C0E9444296C157D0597
:1044B0008E059F0530F48BE00E94692A892BA1F3B9
:1044C00064C08BE00E94692A892B09F05EC080EDF0
:1044D00097E00E94A8070E9444296B017C01D0E06C
:1044E000C1E088E4880E86E2981EA11CB11C11E090
:1044F0008BE00E94692A892B21F58C149D04AE045F
:10450000BF0430F480ED97E00E94A807D1E0F0CF1F
:104510000E9444296C197D098E099F09693C710527
:104520008105910528F30E9444296B017C01C12774
:1045300019F080ED97E002C080E090E00E94A807AB
:10454000D7CF80E090E00E94A807DD23B9F08091EA
:10455000D50590E0019665E070E00E94942E80936E
:10456000D5050E94290D0E94A9130E94480D64EFF1
:1045700071E080E090E00E94732909C080E00E9411
:10458000DF060E94C0110E943F0D0E949821DF911A
:10459000CF911F91FF90EF90DF90CF90BF90AF90A1
:1045A0009F908F900895CF92DF92EF92FF9280E0DC
:1045B0000E94DA070E94B10761E08DE00E94FD29A8
:1045C00061E08CE00E94FD2960E08BE00E94FD2903
:1045D00060E085E00E94FD2961E085E00E94362AC6
:1045E00060E086E00E94FD2961E086E00E94362AB4
:1045F00060E083E00E94FD2961E083E00E94362AAA
:1046000061E08EE00E94FD2960E08EE00E94362A83
:104610000E949F0740E052EC61E070E084EE95E07C
:104620000E94982D0E94A9130E94480D0E94921387
:104630008FEF8093A8040E94C60778940E944429B3
:104640006B017C018091A8048F3F59F40E9444299A
:104650006C197D098E099F09603D774081059105A0
:1046600088F380ED97E00E94A80761E08BE00E944C
:10467000362A2D9A84EE95E00E94502C892B29F041
:1046800084EE95E00E947D2CF5CF6DEF72E084EE14
:1046900095E00E940B2B88E893E00E94300C64E1C7
:1046A00073E084EE95E00E940B2B4AE050E062E05C
:1046B00070E084EE95E00E94DB2B62E370E080E026
:1046C00090E00E94732984EE95E00E94502C04979C
:1046D0000CF184EE95E00E947D2C82349105D1F49A
:1046E00084EE95E00E947D2C8E34910599F484EE41
:1046F00095E00E947D2C8434910561F484EE95E070
:104700000E947D2C819731F480E090E00E94A80700
:104710000E9498214091790550917A0560917B051E
:1047200070917C05DB01CA010197A109B1090497C9
:10473000A105B10568F44093A704433029F440EA89
:1047400056E861E070E004C040E052EC61E070E0E7
:1047500084EE95E00E94982D0E942D222D9880E0F5
:1047600090E00E94A8070E9492131092C7048091C3
:10477000C10583FF11C080918D05882351F0809180
:104780009405882331F080919B05882311F087E000
:1047900001C085E08093C70480E00E947E0A80917A
:1047A000C8040E94B2090E94590B10923F04109253
:1047B0003E0410923D04F12C8091D6058F15B0F087
:1047C00062E370E080E090E00E94732980ED97E062
:1047D0000E94A80762E370E080E090E00E947329E5
:1047E00080E090E00E94A807F394E6CF8091A005B6
:1047F00084FF08C0982F987181E0983109F080E01B
:104800000E947C118FE00E94DA07FF90EF90DF900A
:10481000CF900895EF92FF920F931F93CF93DF9362
:104820008C016EE770E084EE95E00E945906E80185
:10483000F12CF0E2EF2E8E0188818D57823048F402
:104840006DE770E084EE95E00E94590688818E2520
:1048500088832196F801608184EE95E00E94AA2C5D
:10486000F394F9E0FF12E7CF6EE770E084EE95E095
:104870000E945906CDB7DEB7E6E00C94112FA9E0EF
:10488000B0E0E5E4F4E20C94F92E9091C9049111A2
:104890000EC09EEF99838A836B8350E055954795B0
:1048A0004C832D83198618861F821E822EC040914C
:1048B000CE04842F90E0B4E095958795BA95E1F702
:1048C000242F2F7030E08217930719F18DEF898321
:1048D0001B82FE01349650E0842F90E0A4E0959571
:1048E0008795AA95E1F7242F2F7030E08217930760
:1048F00049F0DC01A153BB4F8C918193405F5F5F16
:10490000563051F74093CE045A83CE0101960E944F
:104910000A248091C90490E0019666E070E00E944C
:10492000942E8093C9042996E2E00C94152FA0E000
:10493000B0E0EDE9F4E20C94F22E6C016EE770E069
:1049400084EE95E00E9459068601E12CF12CC0E02E
:10495000D0E030E2B32EF801608183E8860F823028
:1049600078F46DE770E084EE95E00E945906F80156
:1049700060816B2570E084EE95E00E94590604C0CA
:1049800084EE95E00E94AA2CE114F10459F0F8019C
:1049900080819E01280F311DC901C92FDD27C80F55
:1049A000D91FDD273FEFE31AF30A89E0E816F10487
:1049B00059F028E0E216F10421F48C2F8095F601DD
:1049C00080870F5F1F4FC7CFCDB7DEB7E9E00C94EC
:1049D0000E2FA9E0B0E0EFEEF4E20C94F92EE82FF0
:1049E000362F8091C90490E0019664E270E00E9445
:1049F000942E8093C90458E9598350E15A83813039
:104A000089F048F08230B9F08330D9F48B8381EF9C
:104A10008C833D8319C085E08B8381EF8C832F5F6E
:104A20002D8312C08B8381EF8C8384E6489FA00185
:104A300011245D8309C084E08B8381EF8C83ED8337
:104A400003C00E94B91104C0CE0101960E949724B0
:104A50002996E2E00C94152FA2E0B0E0E2E3F5E243
:104A60000C94EE2E182F762E2A8349830E9450290B
:104A70006B017C018091DF048090CA049090CB048C
:104A8000A090CC04B090CD042A8149818823C1F044
:104A9000D701C60188199909AA09BB094C015D0112
:104AA00091EE89169EE29906A104B10420F1241723
:104AB00008F4422F202F672D812F0E94E92413C074
:104AC000D701C60188199909AA09BB094C015D01E2
:104AD00091E3891695E79906A104B10460F0672D6A
:104AE000812F0E943F24C092CA04D092CB04E0924E
:104AF000CC04F092CD042296EDE00C940A2FA2E2B1
:104B0000B0E0E5E8F5E20C94EF2E8CE00E94990904
:104B100081110DC06CE173E084EE95E00E943C2BA6
:104B20002D9A80E00E947E0A0E94590B2D9884EEF7
:104B300095E00E94502C892B01F184EE95E00E94B3
:104B40007D2C9091A704992319F00E94E513EFCFD3
:104B500040913E0450E09A012F5F3F4F2F71332761
:104B600060913F0470E02617370709F3FA01E75B0D
:104B7000FB4F808320933E04DACF8091750584300B
:104B800009F086C00E9450296115710581059105C3
:104B900049F06093B9047093BA048093BB04909376
:104BA000BC040CC081E090E0A0E0B0E08093B904C8
:104BB0009093BA04A093BB04B093BC048091AB045F
:104BC0009091AC0481609093AC048093AB0483E03B
:104BD000809375058FE70E94770909E614E00E942B
:104BE0008A09F80181938F01F4E002371F07B9F7B2
:104BF0002091720480916904982F922796FF3BC000
:104C000090E4922790937204982F98739833F1F45C
:104C100010E0212F30E080916904877090E08217C6
:104C200093074CF11F5F2091A005812F90E0FC01BC
:104C3000E759FB4F24FF04C080810E949B11E9CFFC
:104C4000608184EE95E00E94AA2CE3CF8F7399F4E3
:104C500080916A048093B40480916B048093B204C1
:104C600080916C048093B10480916F0490E09093E4
:104C7000AA048093A90480913D04813019F482E054
:104C800080933D0480913D04833011F410923D04E3
:104C90000E9450296B017C018091AD049091AE047B
:104CA000A091AF04B091B0040097A105B105C9F07F
:104CB000A7019601281B390B4A0B5B0BDA01C901CE
:104CC000883B9B40A105B10560F00E94C809809314
:104CD000B3041092AD041092AE041092AF0410927F
:104CE000B0048091BD049091BE04A091BF04B09126
:104CF000C00446015701881A990AAA0ABB0A88E724
:104D000095E00E94F40786169706A806B90608F4EF
:104D1000B1C0C092BD04D092BE04E092BF04F09234
:104D2000C0040E9457068091A8048830A0F08091AA
:104D3000C1059091C205A091C305B091C4055CE185
:104D4000B695A795979587955A95D1F7892B8A2B74
:104D50008B2B09F0C4C18091A8048F5F8093A804B5
:104D60008091B9049091BA04A091BB04B091BC04A5
:104D70000097A105B105F1F0C81AD90AEA0AFB0AA1
:104D800088E795E00E94F4076C157D058E059F0568
:104D900008F01BC18091C10584FD04C080ED97E03F
:104DA0000E94A8071092B9041092BA041092BB0492
:104DB0001092BC0490917204907C90937204509174
:104DC0003E0480913F0420913D04581709F41AC114
:104DD000223009F017C1905890937204E091A00519
:104DE000E770F0E0E658FC4F6081693008F0F2C0EF
:104DF000615040E04613F0C080933F0487E3840F86
:104E000090917204892B809372044093400483E054
:104E100080933D042C9A109185058091C7048111DF
:104E20003EC18091C10582FD46C1812F0E94790A51
:104E30008091C8040E94B209E091A005E770F0E0FB
:104E4000E658FC4F608182E794E00E94940B8091C9
:104E5000C10582FD39C1E091C804EF5FE093C80449
:104E6000E83109F439C1F0E0E858FA4F8785882322
:104E700009F432C10E94030C813069F58091A005CC
:104E8000887149F18091AB049091AC04880F991F0F
:104E90009093AC048093AB0483E0809375050E94EB
:104EA000590B0E9450296093AD047093AE04809317
:104EB000AF049093B004672B682B692B61F481E0F9
:104EC00090E0A0E0B0E08093AD049093AE04A09396
:104ED000AF04B093B0048091A00584FF2BC08091F3
:104EE000B9049091BA04A091BB04B091BC04892B81
:104EF0008A2B8B2BF9F08091AB049091AC048E7FC0
:104F00000E942A09182F6091A9048091B4040E947C
:104F1000DB13482F612F8091B30449A30E94DB1358
:104F20000091D605282F49A16091B1048091B20467
:104F30000E942C252C988091C5048130C1F018F076
:104F40008230B1F1D9C08BE00E94692A892B09F027
:104F5000D3C081E08093C5040E9444296093C104BA
:104F60007093C2048093C3049093C404C5C08BE0C3
:104F70000E94692A892B31F50E944429C090C104FE
:104F8000D090C204E090C304F090C4046C197D0971
:104F90008E099F09693E73408105910508F4ACC0F4
:104FA00082E08093C50480ED97E00E94A807A4C02A
:104FB0008BE00E94692A892B09F49EC080E090E072
:104FC0000E94A8071092C50497C080E090E00E945C
:104FD000A807F0CE68E00DCF851709F40DCF4F5F1D
:104FE000242F30E090E0F901EE58FB4FDC01A75B85
:104FF000BB4F7C917083F901E05CFB4F708301969D
:105000008F71F8CE2430B1F42091400481E494E013
:10501000A3E7B4E0FC013E2F381B321718F431919E
:105020003D93F9CF87E3820F90917204892B80938F
:105030007204EDCE8091C504823051F4916090935A
:1050400072042D9A8E010F5F1F4FF12CB80110C012
:105050002D9880913D04811103C081E080933D042F
:1050600080913D04833071F784E080933D04EACF62
:105070008F2D69A37AA30E940416F801819391935E
:105080008F01F39469A17AA1F0E1FF12F1CF809131
:10509000A00543E754E087700E947908BBCE112336
:1050A00009F4BFCE9091C60421E0290F2093C604D5
:1050B0009813B7CE1DC085E00E94692A892B09F09C
:1050C000B4CE2D9A17E0B1CE85E00E94692A892BD3
:1050D00009F0C1CE2D98BFCE1092C804CBCE8091DE
:1050E000A804883009F42D9A89E08093A804C2CEE0
:1050F0001092C604115095CEA296ECE00C940B2FA2
:105100008230E8F4E82FF0E0EE0FFF1FE952FA4F8B
:1051100071836083813041F0809169008C7F842BA2
:1051200080936900E89A089580916900440F551FA3
:10513000440F551F837F842B80936900E99A08955B
:105140001F920F920FB60F9211242F933F934F93FC
:105150005F936F937F938F939F93AF93BF93EF93DF
:10516000FF938091D7059091D805892B29F0E09184
:10517000D705F091D8050995FF91EF91BF91AF91B7
:105180009F918F917F916F915F914F913F912F915F
:105190000F900FBE0F901F9018951F920F920FB691
:1051A0000F9211242F933F934F935F936F937F93AD
:1051B0008F939F93AF93BF93EF93FF938091D90504
:1051C0009091DA05892B29F0E091D905F091DA0563
:1051D0000995FF91EF91BF91AF919F918F917F9131
:1051E0006F915F914F913F912F910F900FBE0F9054
:1051F0001F9018951F920F920FB60F9211242F93A4
:105200003F938F939F93AF93BF938091DC059091D1
:10521000DD05A091DE05B091DF053091DB0523E0CF
:10522000230F2D3720F40196A11DB11D05C026E8DE
:10523000230F0296A11DB11D2093DB058093DC0591
:105240009093DD05A093DE05B093DF058091E00526
:105250009091E105A091E205B091E3050196A11DB1
:10526000B11D8093E0059093E105A093E205B09312
:10527000E305BF91AF919F918F913F912F910F9037
:105280000FBE0F901F9018952FB7F8946091DC0512
:105290007091DD058091DE059091DF052FBF0895A7
:1052A0003FB7F8948091E0059091E105A091E20567
:1052B000B091E30526B5A89B05C02F3F19F00196D4
:1052C000A11DB11D3FBF6627782F892F9A2F620F2E
:1052D000711D811D911D42E0660F771F881F991F68
:1052E0004A95D1F70895CF92DF92EF92FF92CF9334
:1052F000DF936B017C010E945029EB01C114D104A2
:10530000E104F10479F00E9450296C1B7D0B683E8A
:105310007340A0F381E0C81AD108E108F108C85130
:10532000DC4FECCFDF91CF91FF90EF90DF90CF90EB
:105330000895789484B5826084BD84B5816084BD0D
:1053400085B5826085BD85B5816085BDEEE6F0E0FE
:10535000808181608083E1E8F0E01082808182605A
:105360008083808181608083E0E8F0E080818160DB
:105370008083E1EBF0E0808184608083E0EBF0E00B
:10538000808181608083EAE7F0E0808184608083AF
:105390008081826080838081816080838081806859
:1053A00080831092C1000895833081F028F4813009
:1053B00099F08230A1F008958630A9F08730B9F0D5
:1053C0008430D1F4809180008F7D03C08091800073
:1053D0008F7780938000089584B58F7702C084B55D
:1053E0008F7D84BD08958091B0008F7703C0809138
:1053F000B0008F7D8093B0000895CF93DF9390E04D
:10540000FC01ED50F44F2491FC01E95FF34F8491CE
:10541000882349F190E0880F991FFC01E15DF34F6B
:10542000A591B4918B5D934FFC01C591D4919FB729
:10543000611108C0F8948C91209582238C93888107
:1054400082230AC0623051F4F8948C91322F309547
:1054500083238C938881822B888304C0F8948C9159
:10546000822B8C939FBFDF91CF910895A1E0B0E094
:10547000ECE3FAE20C94F72E282F30E0F901E15228
:10548000F44F8491F901ED50F44F1491F901E95F63
:10549000F34F04910023C9F0882321F069830E940F
:1054A000D4296981E02FF0E0EE0FFF1FEB5DF34F91
:1054B000A591B4919FB7F8948C91611103C0109598
:1054C000812301C0812B8C939FBF2196E4E00C9433
:1054D000132FCF93DF93282F30E0F901E152F44FDF
:1054E0008491F901ED50F44FD491F901E95FF34F44
:1054F000C491CC2391F081110E94D429EC2FF0E0CB
:10550000EE0FFF1FE55EF34FA591B4912C912D2373
:1055100081E090E021F480E002C080E090E0DF9143
:10552000CF9108958E3008F08E50877020919D01A4
:1055300090E4299F90011124822B80937C0080911C
:105540007A00806480937A0080917A0086FDFCCF97
:10555000809178002091790090E0922B0895A0E04E
:10556000B0E0E5EBFAE20C94F32E6C017A01EB016A
:10557000E60EF71E00E010E0CE15DF0561F0699140
:10558000D601ED91FC910190F081E02DC6010995C5
:10559000080F191FF1CFC801CDB7DEB7E8E00C94B2
:1055A0000F2F6115710589F0DB010D900020E9F7DF
:1055B000AD0141505109461B570BDC01ED91FC91A7
:1055C0000280F381E02D0995089580E090E0089530
:1055D000EF92FF920F931F93CF93DF938C01FB0108
:1055E000C0E0D0E064917F018FEFE81AF80A6623EB
:1055F00061F0D801ED91FC910190F081E02DC8019E
:105600000995C80FD91FF701EDCFCE01CDB7DEB791
:10561000E6E00C94112F0E94D12A0895DC01ED914F
:10562000FC910190F081E02D099508950F931F934F
:10563000CF93DF93EC016DE00E940E2B8C016AE0AA
:10564000CE010E940E2B800F911FDF91CF911F91F1
:105650000F9108950F931F93CF93DF93EC010E9456
:10566000E82A8C01CE010E94162B800F911FDF913A
:10567000CF911F910F9108950F931F93CF93DF93B5
:10568000EC010E94D12A8C01CE010E94162B800FC2
:10569000911FDF91CF911F910F9108950F931F9349
:1056A000CF93DF93EC010E940E2B8C01CE010E9460
:1056B000162B800F911FDF91CF911F910F910895AD
:1056C000A1E2B0E0E6E6FBE20C94EF2E7C01C42EF2
:1056D000E52FCB01D22E19A221E02D1510F02AE0E2
:1056E000D22E8E010F5D1F4F8D2C912CA12CB12C31
:1056F0006C2D7E2FA50194010E94A82E8C2DD29E88
:1057000080191124015011098A3010F4805D01C004
:10571000895CF8018083211531054105510521F08F
:10572000C22EE32FCA01E4CFB801C7010E94D12ADB
:10573000A196ECE00C940B2FA0E0B0E0E2EAFBE2D3
:105740000C94F32EEC016A017B012115310541F423
:10575000E881F9810190F081E02D642F09951DC049
:105760002A303105A9F477FF12C06DE20E940E2B9A
:105770008C0144275527BA014C195D096E097F0930
:105780002AE0CE010E94602B800F911F06C02AE004
:10579000B701A601CE010E94602BCDB7DEB7E8E0CD
:1057A0000C940F2F9A01AB01662757FD6095762F59
:1057B0000E949C2B08950F931F93CF93DF93EC01CE
:1057C0009A01AB01662757FD6095762F0E949C2BAE
:1057D0008C01CE010E94162B800F911FDF91CF917B
:1057E0001F910F9108952115310549F4DC01ED91C8
:1057F000FC910190F081E02D642F099508950E949D
:10580000602B08959A01462F50E060E070E00E94FE
:10581000F32B08959A01AB0160E070E00E94F32B36
:1058200008950F931F93CF93DF93EC010E94F32B06
:105830008C01CE010E94162B800F911FDF91CF911A
:105840001F910F9108950F931F93CF93DF93EC0156
:105850009A01AB0160E070E00E94F32B8C01CE0155
:105860000E94162B800F911FDF91CF911F910F91F6
:1058700008950F931F93CF93DF93EC019A01462F66
:1058800050E060E070E00E94F32B8C01CE010E949A
:10589000162B800F911FDF91CF911F910F910895CB
:1058A000FC0124853585F901E05CFF4F8081918101
:1058B000F901EE5BFF4F20813181821B930B8F73C7
:1058C00099270895FC0184859585FC01E05CFF4FD4
:1058D00040815181FC01EE5BFF4F208131814217F5
:1058E000530741F00190F081E02DE80FF91F80810E
:1058F00090E008958FEF9FEF0895FC0184859585D2
:10590000FC01E05CFF4F40815181FC01EE5BFF4FE9
:10591000208131814217530779F0A081B181A80F0E
:10592000B91F8C91208131812F5F3F4F2F73332717
:105930003183208390E008958FEF9FEF0895FC015D
:1059400081A1882329F0A489B5898C9186FFFBCF9A
:1059500011A20895CF93DF93FC0126853785D901E5
:10596000A05CBF4F8D919C91119701968F739927E1
:10597000E901CE5BDF4F4881598184179507D9F340
:105980000D90BC91A02DA20FB31F6C93A685B78577
:10599000A05CBF4F11969C938E93A689B7892C91DA
:1059A00081E090E0078C02C0880F991F0A94E2F70B
:1059B000282B2C9381E081A30488F589E02D808138
:1059C0008064808381E090E0DF91CF910895089515
:1059D0001F920F920FB60F9211242F933F934F9364
:1059E0008F939F93EF93FF938091C00082FD1CC023
:1059F0004091C60080918A0690918B0601968F7324
:105A0000992720918C0630918D068217930771F0AB
:105A1000E0918A06F0918B06E65BF94F4083909304
:105A20008B0680938A0602C08091C600FF91EF9199
:105A30009F918F914F913F912F910F900FBE0F909B
:105A40001F90189584EE95E00E94502C892B11F040
:105A50000E94E72C08951F920F920FB60F92112407
:105A60002F933F938F939F93EF93FF93209146063D
:105A700030914706809148069091490628173907CA
:105A800031F48091C1008F7D8093C10014C0E091FA
:105A90004806F0914906EA5FF94F20818091480657
:105AA0009091490601968F739927909349068093A8
:105AB00048062093C600FF91EF919F918F913F91EF
:105AC0002F910F900FBE0F901F901895A0E0B0E09F
:105AD000ECE6FDE20C94EF2EFC011382128288EEBC
:105AE00093E0A0E0B0E084839583A683B7838CEB3A
:105AF00093E0918380837587648757874687318BCE
:105B0000208B138B028BF58AE48AD78AC68AB18EE2
:105B1000A08E938E828E8F85848F8889858F8989C8
:105B2000868F8A89878F8B8980A3ECE00C940B2F5A
:105B3000CF92DF92EF92FF92CF93DF93EC016A0155
:105B40007B01411581EE580761057105F9F0EC897B
:105B5000FD8981E090E008A002C0880F991F0A9497
:105B6000E2F7808360E079E08DE390E0A7019601A1
:105B70000E94A82E21503109410951095695479597
:105B800037952795211580E1380798F0EC89FD8934
:105B9000108260E874E88EE190E0A70196010E940F
:105BA000A82E21503109410951095695479537953D
:105BB0002795E889F9893083EA89FB89208319A22E
:105BC000EE89FF89408181E090E09C010C8C02C04D
:105BD000220F331F0A94E2F7422B4083EE89FF899C
:105BE00040819C010D8C02C0220F331F0A94E2F702
:105BF000422B4083EE89FF8940819C010E8C02C0BC
:105C0000220F331F0A94E2F7422B4083EE89FF896B
:105C100020810F8C02C0880F991F0A94E2F78095AB
:105C200082238083DF91CF91FF90EF90DF90CF9020
:105C300008958F929F92AF92BF92CF92DF92EF9290
:105C4000FF920F931F9381E08F9385E08F9387E0FE
:105C50008F9383E08F9384E08F93E6EC8E2E912CCC
:105C6000F2ECAF2EB12CA1ECCA2ED12CB0ECEB2E65
:105C7000F12C04EC10E025EC30E046E056E06AE45C
:105C800076E084EE95E00E94662D0F900F900F90C5
:105C90000F900F901F910F91FF90EF90DF90CF909A
:105CA000BF90AF909F908F9008950E9499290E9475
:105CB000D322C2E2DDE20E947F252097E1F30E9419
:105CC000222DF9CFA29FB001B39FC001A39F700DF9
:105CD000811D1124911DB29F700D811D1124911DF4
:105CE00008950E94622EA59F900DB49F900DA49FD1
:105CF000800D911D11240895B7FF0C94712E0E9400
:105D0000712E821B930B0895DB018F939F930E944A
:105D1000712EBF91AF91A29F800D911DA39F900DF9
:105D2000B29F900D1124089597FB072E16F400944E
:105D300007D077FD09D00E94262F07FC05D03EF43E
:105D4000909581959F4F0895709561957F4F089527
:105D5000A1E21A2EAA1BBB1BFD010DC0AA1FBB1F6F
:105D6000EE1FFF1FA217B307E407F50720F0A21BE1
:105D7000B30BE40BF50B661F771F881F991F1A944E
:105D800069F760957095809590959B01AC01BD0178
:105D9000CF010895052E97FB1EF400940E94E12E7A
:105DA00057FD07D00E94A82E07FC03D04EF40C9498
:105DB000E12E50954095309521953F4F4F4F5F4FC5
:105DC000089590958095709561957F4F8F4F9F4F67
:105DD00008952F923F924F925F926F927F928F928F
:105DE0009F92AF92BF92CF92DF92EF92FF920F936A
:105DF0001F93CF93DF93CDB7DEB7CA1BDB0B0FB674
:105E0000F894DEBF0FBECDBF09942A883988488830
:105E10005F846E847D848C849B84AA84B984C884C6
:105E2000DF80EE80FD800C811B81AA81B981CE0FBD
:105E3000D11D0FB6F894DEBF0FBECDBFED010895A2
:105E4000EE0FFF1F0590F491E02D0994AA1BBB1BD8
:105E500051E107C0AA1FBB1FA617B70710F0A61B6A
:105E6000B70B881F991F5A95A9F780959095BC018B
:105E7000CD0108958F929F92AF92BF92CF92DF9201
:105E8000EF92FF92CF93DF93EC01688179818A8151
:105E90009B81611571058105910521F464E279ED1D
:105EA0008BE597E02DE133EF41E050E00E94CA2EF0
:105EB00049015A019B01AC01A7EAB1E40E94712E8D
:105EC0006B017C01ACEEB4EFA50194010E947F2E22
:105ED000C60ED71EE81EF91EF7FE06C081E0C81ADE
:105EE000D108E10880E8F80AC882D982EA82FB82F8
:105EF000C701B6019F77DF91CF91FF90EF90DF90C0
:105F0000CF90BF90AF909F908F9008950E943A2FAE
:105F1000089586E091E00E943A2F0895609306016B
:105F200070930701809308019093090108952F92BF
:105F30003F925F926F927F928F929F92AF92BF92A9
:105F4000CF92DF92EF92FF920F931F93CF93DF9345
:105F50008B01EA016115710521F0DB018C9311962B
:105F60009C93209739F09E0122503109233231054C
:105F700008F0D8C07C016701BFEFCB1ADB0A5601DD
:105F8000F7016080862D90E00E94C930892B11F0C6
:105F90007601F1CFFDE26F120AC0570182E0A80E30
:105FA000B11CD70111966C90772473940BC0BBE29F
:105FB0006B1207C05701E2E0AE0EB11CD70111967B
:105FC0006C90712CCE018F7E892B89F4B0E36B121B
:105FD00037C0F50180818F7D8835D1F46180F2E092
:105FE000AF0EB11C872D8260782EC0E1D0E0CA30A0
:105FF000D10551F1C031D10521F0C830D10599F456
:1060000009C0CC24CA94DC2CEC2CAFE0FA2E22C0C0
:10601000209769F7C8E0D0E0CC24CA94DC2CEC2CA3
:10602000FFE1FF2E17C06FEF7FEFCB019E014427EA
:1060300037FD4095542F0E94A82E69017A010AC0AD
:106040002097A9F6CAE0D0E0E9E9CE2EDC2CEC2CB2
:10605000E9E1FE2EF50160E020E030E0A9014E010B
:10606000AA2497FCA094BA2C1F0170ED572E560C51
:10607000A9E0A51570F48FEB860D8A3118F499EC20
:10608000592E06C08FE9860D8A3148F589EA582EC7
:10609000560C852D90E08C179D070CF56F3FD9F0BD
:1060A000C216D306E406F50698F0C501B4010E94B5
:1060B000842E9B01AC01852D90E0A0E0B0E0280F7C
:1060C000391F4A1F5B1F281739074A075B0710F45F
:1060D0006FEF01C061E03196D1016C90C5CF011521
:1060E000110551F0662311F0319703C071FE04C011
:1060F0003297D801ED93FC9370FE07C05095409500
:10610000309521953F4F4F4F5F4F67FF10C082E2A0
:1061100090E090938F0680938E066FEF7FEF8FEF66
:106120009FEF07C060E070E080E090E002C0B9013E
:10613000CA01DF91CF911F910F91FF90EF90DF90F7
:10614000CF90BF90AF909F908F907F906F905F9017
:106150003F902F900895FC0188279927E89421917A
:106160002032E9F3293010F02E30C8F32B3241F001
:106170002D3239F4689404C00E94FD30820F911DC5
:10618000219120532A30C0F31EF4909581959F4FA2
:106190000895911150C0803219F089508550D0F780
:1061A000089548EC53E00E94D6300895FA01A19179
:1061B000B081009719F41097E1F0CD01DC01CD0119
:1061C0000D90002011F4C00113C0FB012191222386
:1061D00019F02015D9F7F3CFFB012191201519F4FF
:1061E0001E92119606C02223C1F70D900020A1F740
:1061F000D001FA01A193B08308957AE0979F902D82
:10620000879F802D910D11240895F999FECF92BD9D
:1062100081BDF89A992780B50895262FF999FECF68
:106220001FBA92BD81BD20BD0FB6F894FA9AF99AB3
:106230000FBE01960895992788270895F894FFCFF7
:1062400000009006200001000000FF000200020094
:10625000020002000200020002000200020002002E
:106260000200020002000200020002802500000578
:10627000400AA1204EA50020244EA52C2330C01298
:1062800000001A400AA1204EA5001B1E27522C23F5
:10629000308025000005400AA1204EA50020244E94
:1062A000A52C2330004B000006400AD0009D490079
:1062B0007B289D492C233000E1000005400A450160
:1062C000D7DC03B81E0EBF00232E48E801008A4029
:1062D0000A6001555502AD1E20000023C801545824
:1062E0002074696D656F75742100596573004E6F78
:1062F000002C00386368004E2F41002C205B005DAD
:106300002028002900486F70206368616E6E656CFC
:10631000200020402000456E746572696E67206120
:1063200064617074697665206368616E6E656C2067
:1063300073656C656374696F6E2C207069636B693B
:106340006E673A007363616E6E6572206D6F64658F
:10635000004E4F5420454E41424C45440053656E1B
:1063600064696E672073657474696E677320746FF7
:106370002052580A00526573657474696E67207301
:10638000657474696E6773206F6E2052580A0041FD
:10639000626F727465642065646974730A00696E63
:1063A00076616C69642073656C656374696F6E00F7
:1063B0000D0A496E76616C696420696E707574208F
:1063C0002D206469736361726465642107005365FD
:1063D0007474696E677320736176656420746F20CE
:1063E000454550524F4D0A0052657665727465649A
:1063F0002073657474696E67732066726F6D2045D3
:106400004550524F4D0A004C6F61646564206661CF
:1064100063746F72792064656661756C74730A00C9
:106420004B657920616E64206368616E6E656C7384
:106430002072616E646F6D697A65640A004F7065E1
:106440006E4C52536E672054582073746172746995
:106450006E672000206F6E20485720006D6F6475B6
:106460006C65206C6F636B65643F00342B340038BF
:1064700000382B340031320031322B3400313600F9
:1064800050504D0052535349005344410053434C24
:1064900000525844005458440041494E004C424573
:1064A00045500053504B54524D00534255530053E6
:1064B000554D44004C4C494E440000070B0C101144
:1064C0001500B7012B032F033103350338033D03B8
:1064D000B7014003440349034D03510355035903D6
:1064E0005D0363036A036F0374038D028D028D02E3
:1064F0008D02160A1322312900000000AA2CAF2AAF
:08650000502C7D2C622C9F2C15
:107E00000F92CDB7DEB7112484B714BE81FFF1D035
:107E100082E08093C00088E18093C10086E0809377
:107E2000C20080E18093C4008EE0CDD088249924E4
:107E3000CC24C394F5E0DF2EE1E1EE2E73E0F72EC3
:107E4000B6D0082F813479F4B2D08983C2D0898129
:107E5000823811F481E005C0813811F485E001C059
:107E600083E09ED09AC0823411F484E103C085344B
:107E700019F485E0B6D091C0853561F498D0082F0B
:107E800010E095D090E0982E8824802A912A880CC2
:107E9000991C82C0863521F484E0A3D080E0E1CF34
:107EA000843609F04CC083D082D0A82E80D0B82E62
:107EB00000E011E07CD0F80181938F01AE16D1F77C
:107EC00088D0FB2DF53489F4E0E0F1E00BC0F9999E
:107ED000FECF92BC81BC0894811C911C819180BD15
:107EE000FA9AF99AEA1598F358C08B2D863409F05E
:107EF00054C0F401F7BEE89507B600FCFDCFF401CD
:107F0000A0E0B1E02C9130E011968C91119790E0B7
:107F1000982F8827822B932B12960C01C7BEE895C9
:107F20001124329681E0A038B80761F7F401D7BE7A
:107F3000E89507B600FCFDCFE7BEE8952EC0843774
:107F4000F1F435D034D0182F32D0B82E42D0FB2DDA
:107F5000F63421F4F40105914F010CC0FB2DF534EA
:107F600049F4F999FECF92BC81BC0894811C911C04
:107F7000F89A00B5802F14D0115049F70EC08537FC
:107F800039F427D08EE10CD085E90AD08FE069CF93
:107F9000813511F488E017D01CD080E101D050CF9A
:107FA0009091C00095FFFCCF8093C600089580910A
:107FB000C00087FFFCCF8091C00084FD01C0A89560
:107FC0008091C6000895E0E6F0E098E19083808318
:107FD0000895EDDF803219F088E0F5DFFFCF84E10E
:107FE000DFCF1F93182FE3DF1150E9F7F2DF1F9166
:0E7FF0000895282E80E0E7DFEE27FF27099492
:027FFE0001057B
:0400000300007E007B
:00000001FF
